:100000000C9443180C946B180C946B180C946B188C
:100010000C946B180C946B180C946B180C946B1854
:100020000C946B180C946B180C946B180C946B1844
:100030000C946B180C946B180C946B180C946B1834
:100040000C946B180C946B180C946B180C946B1824
:100050000C946B180C946B180C946B180C94C32FA5
:100060000C946B180C946B180C946B180C946B1804
:100070000C946B180C946B180C946B180C946B18F4
:100080000C940D300C946B180C946B180C946B182A
:100090000C946B180C946B180C946B180C946B18D4
:1000A0000C946B180C946B180C946B18D5F08D1481
:1000B000A1C881CFD9F1AF200045120445140445F1
:1000C0001604451804451A04451C04451E04452021
:1000D00004452204452404452604452804452A04F1
:1000E000452C04452E044530044532044534044370
:1000F00034014134013F34013D3501393501373593
:10010000013535013336013136012F36012D3601E7
:100110002B36992C13042C15042C17042C19042CA1
:100120001B042C1D042C1F042C21042C23042C251F
:10013000042C27042C29042C2B042C2D042C2F04F4
:100140002C31042C33042C35012C3701293701279D
:1001500037012537012337011F38011D38011B38AE
:1001600001193801173801153999121304121504B1
:10017000121704121904121B04121D04121F041278
:100180002104122304122504122704122904122B1D
:1001900004122D04122F04123104123304123504F8
:1001A0001237041239011139010F39010D39010BD0
:1001B0003A01093A01073A01053A01033A01013BC4
:1001C00001FF3D01FF3F01FF4101FF4301FF4501E9
:1001D000FF4701FF4901FF4B01FF4D01FF4F01FFA9
:1001E0005101FF5301015302035302055302075308
:1001F000020954020B54020D54020F54021154020E
:100200001355021555021755021955021B55021DAB
:1002100056021F5602215602235602255602275720
:10022000022957022B57022D57022F57023158022D
:100230003358023558023758023958023B59023DAB
:1002400059023F5902415902435902455A02475A3D
:1002500002495A024B5A024D5A024F5B02515B024D
:10026000535B02555B02575B02595C025B5C025DAB
:100270005C025F5C02615C02635D02645E02655F5A
:100280000265610265630265650265670265690270
:10029000656B02656D02656F0265710265730263CD
:1002A00073016173015F73015D74015B74015974C3
:1002B000015774015574015375015175014F750152
:1002C0004D75014B7501497601477601457601432D
:1002D00076014176013F77013D77013B7701397720
:1002E000013777013578013378013178012F7801B2
:1002F0002D78012B790129790127790125790123AD
:100300007901217A011F7A011D7A011B7A01197A7C
:1003100001177B01157B01137B01117B010F7B0111
:100320000D7C010B7C01097C01077C01057C01032C
:100330007D01017E010180010182010184010186AC
:1003400001018801018A01018C010000040B794A36
:1003500001180D794A001C0F794A000C11784900E8
:100360000C137849000C157849000C177849000CDB
:10037000197849000C1B7748000C1D7748000C1FAA
:100380007748000C217748000C237748000C25762D
:1003900047000C277647000C297647000C2B764740
:1003A000000C2D7647000C2F7546000C3175460069
:1003B0000C337546000C357546000C377546000C3D
:1003C000397445000C3B7445000C3D7445000C3FEE
:1003D0007445001C417445001C437343001C457365
:1003E00043001C477343000C497343000C4B734399
:1003F000000C4D7242000C4F7242000C51724200D0
:100400000C537242000C557242000C577141000CA3
:10041000597141000C5B7141000D5D714100055D3A
:100420006F3F0C035D6D3D0C035D6B3B0D035D6920
:10043000390D035D67370C035D65350C035D633370
:100440000D035D61310D035D5F2F0C035D5D2D0CB0
:10045000035D5B2B0D035D592900465B5929004E56
:10046000595828004C575828004C555828004C53D0
:100470005828004C515828004C4F5727004C4D57D6
:1004800027005C4B5727005C495727005C475727DC
:10049000005C455626005C435626005C415626000B
:1004A0005C3F5626005C3D5626005C3B5525005CB3
:1004B000395525005C375525005C355525005C33E2
:1004C0005525005C315424005C2F5424005C2D54CD
:1004D00024004C2B5424004C295424004C27532333
:1004E000004C255323004C235323004C215323005D
:1004F0004C1F5323004C1D5222004C1B5222004C17
:10050000195222004C175222004C155222004C1353
:100510005121004C115121004C0F5121004C0D5123
:1005200021004D0B512100490B4F1F0C030B4D1D9A
:100530000C030B4B1B0D030B49190D030B47170C39
:10054000030B45150C030B43130D030B41110D0356
:100550000B3F0F0C030B3D0D0C030B3B0B0D030B63
:1005600039090D030B37070C030B35050C030B334F
:10057000030D030B31010D030B2F000C030B2D009A
:100580000C030B2B000D030B29000D030B27000C94
:10059000030D2400002A0D2400000E0F2400000C7F
:1005A000112400000C132400000C152400000C176B
:1005B0002400000C192400000C1B2400000C1D2436
:1005C00000000C1F2400000C212400000C23240038
:1005D000000C252400000C272400000C2924000016
:1005E0000C2B2400000C2D2400000C2F2400000CE8
:1005F000312400000C332400000C352400000C379B
:100600002400000C392400000C3B2400000C3D2485
:1006100000000C3F2400000C412400000C43240087
:10062000000C452400000C472400000C4924000065
:100630008C4B2400008C4D21000B044F1F000B0C31
:10064000511E000B0C531D000B0C551D000F0055C7
:100650001D000F00551D000F00551D000F00551DFA
:10066000000F00551D000F00551D000F005F150005
:100670000F005F15000F005B150013005B150013E2
:10068000005F170014005F170014006419001400C5
:1006900064190014006419001400581D0114005856
:1006A0001D021400581D031400542A041400542A77
:1006B000051400542A061400583207140058320852
:1006C0001400583209140059340900005934090142
:1006D000005B340903005D340905005F340907003D
:1006E00061340909006334090300653409050067B2
:1006F0003409070069340909006B340903006D34BB
:100700000905006F340907007134090900733409C1
:1007100003007534090500773409070079340909A5
:10072000007B340903007D340905007F340907008C
:100730008134090700551E000B00571F010B005B99
:1007400021030B005D23050B005F26080B006129C8
:100750000B0B00632C0E0B006530120B006733157A
:100760001000693315110069331512006933151231
:100770000069331512006933151200693315120030
:100780006933151200693315120069331512004DD3
:1007900024000B004F24000B005124000B005325B4
:1007A000000B005525000B005725010B005B2603AD
:1007B0000B005D26050B005F27080B0061280B0B63
:1007C0000063290E0B00652B120B00672E1510001D
:1007D0006933151100693315120069331512006968
:1007E000331512006933151200693315120069338D
:1007F00015120069331512006933151200C7340948
:100800000100633409010063340900006334090006
:100810000061330902005F310904005D2E09060002
:100820005B2C090800592A090200572809040055C1
:1008300026090600532409080051220902004F210D
:100840000904004D220906004B2409080049240927
:10085000020047240904004524090600432409082E
:100860000041240902003F240904003D2409060038
:100870003B24090800392409020037240904003503
:1008800024090600332409080031240902002F241A
:100890000904002D240906002B2409080029240935
:1008A000020027240904002524090600232409083E
:1008B0000021240902001F240904001D2409060048
:1008C0001B220908001920090200171E0804001540
:1008D0001C070600131A0608001118050A000F1657
:1008E000040A000F14030A000F13020A000F11017B
:1008F0000A000D0F000A000B0E000200090E000492
:1009000000070E000600050E000800030E0002009E
:10091000030E000C00030E000C00030E000D00037C
:100920000E000D00030E000C00030E000C00030E61
:10093000000D00030E000D00030E000C00030E005E
:100940000C00030E000D00030E000D00030E000C42
:1009500000030E000200010E000400FF0E0006005E
:10096000FD0E000800FB0E000200F90E000400F767
:100970000E000600F50E0008007924000004FCFEBD
:10098000FFFFFFFFFFFFFFFFFFFFFFFFFFFFFFFF77
:10099000FFFFFFFFFFFEFEFC070F1F1F1F1F1F1F94
:1009A0001F1F1F1F1F1F1F1F1F1F1F1F1F1F1F1F57
:1009B0001F0F1A0D00FC02FAFAAAAA02F2FA2AF292
:1009C00002B2BAEA6A021AFAE21A02FC000000074E
:1009D000080A0A0A0A080A0A090A080A0A0A090881
:1009E000080A0A080807000000FC02FAFA22FA02C4
:1009F000F2FA2AF202FAFA2AD202FAFA8AF202FC8D
:100A000000000007080A0A090A080A0A090A080A6F
:100A10000A090A080A0A0A0A08070000FCFCFCFC8A
:100A2000FCFCFCFCFCFCFCFCFCFCFCFCFCFFFFFFFD
:100A3000FFFFFFFFFFFFFFFFFFFFFEFCF8010101CB
:100A40000101010101010101010101010101010196
:100A5000010103070F0F0F0F0F0F0F070301210CE9
:100A6000000078281000782850007858001048209E
:100A700000104820000078FC8ED6DAD68EFC780074
:100A80000000000000000000000000000000000066
:100A90000000000000000001020505050505020137
:100AA00000000408022905023E09093E3F25251AD7
:100AB0001E2121123F21211E3F2525213F05050131
:100AC0001E21293A3F04043F213F21001021211F0C
:100AD0003F040A313F2020203F02023F3F02043FF3
:100AE0001E21211E3F0909061E21112E3F0909362C
:100AF00022252519013F01011F20201F0F10201F53
:100B00003F10103F3B04043B03043807312D2321E1
:100B10001E29251E223F2000322929261221251AAE
:100B20000C0A3F08172525191E252518013905032C
:100B30001A25251A0629291EFCFEFFFFFFFFFFFFCD
:100B4000FFFFFFFFFFFFFFFFFFFFFFFFFFFFFFFFB5
:100B5000FFFFFFFFFFFFFFFFFFFFFFFFFFFFFFFFA5
:100B6000FFFFFFFFFFFFFFFFFFFFFFFFFFFFFFFF95
:100B7000FFFFFFFFFFFFFFFFFFFFFFFFFFFFFFFF85
:100B8000FFFFFFFFFFFFFFFFFFFFFFFFFEFEFCFF7A
:100B9000FFFFFFFFFFFFFFFFFFFFFFFFFFFFFFFF65
:100BA000FFFFFFFFFFFFFFFFFFFFFFFFFFFFFFFF55
:100BB000FFFFFFFFFFFFFFFFFFFFFFFFFFFFFFFF45
:100BC000FFFFFFFFFFFFFFFFFFFFFFFFFFFFFFFF35
:100BD000FFFFFFFFFFFFFFFFFFFFFFFFFFFFFFFF25
:100BE000FFFFFFFFFFFF01030707070707070707CF
:100BF0000707070707070707070707070707070785
:100C00000707070707070707070707070707070774
:100C10000707070707070707070707070707070764
:100C20000707070707070707070707070707070754
:100C300007070707070707070707070703571300F3
:100C4000FC0202F2F2F282F2F2F202F2F2F202C2DA
:100C5000E2F2121252624202F2F2F282F2F2F20274
:100C600002E2F29292122202C2E2F23212127222D4
:100C700002C2E2F2125212F2E2C202F2F2F21212D4
:100C8000F2F2E202F2F2F292921202E2F292921284
:100C9000220202FC000000FF00005F5F5F005F5F58
:100CA0005F005F5F5F00172F5F50515F2F5F005F36
:100CB0005F5F005F5F5F002C5C5151535F2E001738
:100CC0002F5F585050582E00172F5F5050505F2FF5
:100CD00017005F5F5F01015F5E58005F5F5F50520A
:100CE000500C5C5151535F2E0000FF0000000102C8
:100CF00002020202020202020202020202020202D4
:100D000002020202020202020202020202020202C3
:100D100002020202020202020202020202020202B3
:100D200002020202020202020202020202020202A3
:100D30000202020202020202020202020202020293
:100D400002010000FFFFFFFFFFFFFFFFFFFFFFFFAC
:100D5000FFFFFFFFFFFFFFFFFFFFFFFFFFFFFFFFA3
:100D6000FFFFFFFFFFFFFFFFFFFFFFFFFFFFFFFF93
:100D7000FFFFFFFFFFFFFFFFFFFFFFFFFFFFFFFF83
:100D8000FFFFFFFFFFFFFFFFFFFFFFFFFFFFFFFF73
:100D9000FFFFFFFFFFFFFFFFFFFFFFFFFFFFFFFF63
:100DA000FFFFFFFFFFFFFFFFFFFFFFFFFFFFFFFF53
:100DB000FFFFFFFFFFFFFFFFFFFFFFFFFFFFFFFF43
:100DC000FFFFFFFFFFFFFFFFFFFFFFFFFFFFFFFF33
:100DD000FFFFFFFFFFFFFFFFFFFFFFFFFFFFFFFF23
:100DE000FFFFFFFFFFFFFFFFFFFFFFFFFFFFFFFF13
:100DF000FFFFFFFFFFFFFFFFFFFFFFFFFFFFFFFF03
:100E0000FFFFFFFFFFFFFFFFFFFFFFFFFFFFFFFFF2
:100E1000FFFFFFFFFFFFFFFFFFFFFFFFFFFFFFFFE2
:100E2000FFFFFFFFFFFFFFFFFFFFFFFFFFFFFFFFD2
:100E3000FFFFFFFFFFFFFFFFFFFFFFFFFFFFFFFFC2
:100E4000FFFFFFFFFFFFFFFFFFFFFFFFFFFFFFFFB2
:100E5000FFFFFFFFFFFFFFFFFFFFFFFFFFFFFFFFA2
:100E6000FFFFFFFF03030303030303030303030362
:100E70000303030303030303030303030303030342
:100E80000303030303030303030303030303030332
:100E90000303030303030303030303030303030322
:100EA000030303030303030303030303482200FCB8
:100EB000060202020202020202020202020202020E
:100EC0000202020202020202020202020202020202
:100ED00002020202020202020202020202020202F2
:100EE00002020202020202020202020202020202E2
:100EF00002020206FC0000FF0000000000000000EB
:100F000000000000000000000000000000000000E1
:100F100000000000000000000000000000000000D1
:100F200000000000000000000000000000000000C1
:100F3000000000000000000000000000FF0000FFB3
:100F400000000000000000000000000000000000A1
:100F50000000000000000000000000000000000091
:100F60000000000000000000000000000000000081
:100F70000000000000000000000000000000000071
:100F800000000000FF0000FF8000000000000000E3
:100F90000000000000000000000000000000000051
:100FA0000000000000000000000000000000000041
:100FB0000000000000000000000000000000000031
:100FC000000000000000000000000080FF000000A2
:100FD0000101010101010101010101010101010101
:100FE00001010101010101010101010101010101F1
:100FF00001010101010101010101010101010101E1
:1010000001010101010101010101010101010101D0
:101010000101010100000B08878F9DB7E7C7A5D725
:10102000AF978D0000000000000000000306080BD1
:101030000E1113FCFEFFFFFFFFFFFFFFFFFFFFFF8F
:10104000FFFFFFFFFFFFFFFFFFFFFFFFFFFFFFFFB0
:10105000FFFFFFFFFFFFFFFFFFFEFC3F7FFFFFFFE4
:10106000FFFFFFFFFFFFFFFFFFFFFFFFFFFFFFFF90
:10107000FFFFFFFFFFFFFFFFFFFFFFFFFFFFFFFF80
:10108000FF7F3F28100000F80404040404E4242433
:10109000C404C42424C404E40404E40444A4244490
:1010A00004E4A4A4240404040404F8000000001FC1
:1010B0002020202020272121202027212127202314
:1010C00024242320222425222027242424202020F5
:1010D00020201F0000FCFEFFFFFFFFFFFFFFFFFFC0
:1010E000FFFFFFFFFFFFFFFFFFFFFFFFFFFFFFFF10
:1010F000FFFFFFFFFFFFFFFFFFFFFFFFFFFFFFFF00
:10110000FFFFFFFFFFFFFFFFFFFFFFFFFFFEFC3FB3
:101110007FFFFFFFFFFFFFFFFFFFFFFFFFFFFFFF5F
:10112000FFFFFFFFFFFFFFFFFFFFFFFFFFFFFFFFCF
:10113000FFFFFFFFFFFFFFFFFFFFFFFFFFFFFFFFBF
:10114000FFFFFFFFFFFFFF7F3F3A100000F804049E
:10115000040404C424A4A404C42424C404E44484CF
:1011600044E404E4A4A424040404C42424C404E43F
:101170000404E404E4A4A42404E42424C40404042F
:101180000404F8000000001F202020202023242435
:10119000232027212127202720202027202724241F
:1011A0002420202023242423202122242320272418
:1011B0002424202721212620202020201F00000475
:1011C0000406090F060A0F0F08090D0F0A090B0F75
:1011D0000F03020F0F070D0D0D0F0A0E0E010D0F5D
:1011E000030E0B0B0F07050F0F143E7E7F7F3F1E74
:1011F0000C080700143C363A160C00FCFEFFFFFFFB
:10120000FFFFFFFFFFFFFFFFFFFFFFFFFFFFFFFFEE
:10121000FFFFFEFC000103030303030303030303B7
:1012200003030303030303030303030100190A0079
:10123000FC02020202020202020202020202020294
:10124000020202020202FC00000001010101010190
:10125000010101010101010101010101010101007F
:1012600000040406090F060A0F0F08090D0F0A09EA
:101270000B0F0F03020F0F070D0D0D0F0A0E0E01BE
:101280000D0F030E0B0B0F07050F0FFCFEFFFFFFEB
:10129000FFFFFFFFFFFFFFFFFFFFFFFFFFFFFFFF5E
:1012A000FEFC3F7FFFFFFFFFFFFFFFFFFFFFFFFF92
:1012B000FFFFFFFFFFFFFF7F3F171000FC0202FA56
:1012C0008202FAAA027A827A02FAAA02FA82020256
:1012D000FC00003F404040404040404040404040D3
:1012E000404040404040403F0040E8FCFCFCFCFCEB
:1012F000DCBBFFFDFFFBB870F0F0F0F070200000E9
:1013000000000000000001010101010103030303CB
:101310000303010000002070F0F0F0F070BBFFFD4F
:10132000FFFBB8DCFCFCFCFCFCE840000001030314
:10133000030303030101010101010000000000009B
:101340000090F8F8F8F8F8F8F8FBFFFFFFFBF8F862
:10135000F8F8F8F8F8F89000010101010101010125
:1013600001010101010101010101010100160A0051
:101370004048586858488890B3D5B390102060A072
:1013800060202000000000000000000000000000BD
:1013900000000101010101010000000000202060A7
:1013A000A060201093B5D3B0908848586858484042
:1013B0000000000001010101010100000000000027
:1013C00000000000000000009090B0D0B09090901D
:1013D000B3D5B3909090B0D0B09090900000000042
:1013E00000000000000000000000000000000000FD
:1013F000000000070B066B9DFBDE0A0000000604E0
:1014000002040000009DFBDE000000000604020054
:1014100000000000FB0000000000000400000000CD
:1014200000000000000000000004000000000000B8
:10143000F8000000000000000000000000000300B1
:10144000000000000000000000080CF4FEFEFFFF9A
:10145000FFFEEC0E0F0F0F0F0F0E0E080CECFEFF31
:10146000FFFFFEFEF40E0E0F0F0F0F0F0E0ADFFF31
:10147000FFFFFF6F040607070706006FFFFFFFFF70
:10148000DF0A00060707070604FFFFFFFFFFFFE66E
:1014900000020707070600E6FFFFFFFFFFFF000649
:1014A00007070702001FFFFFFFFFFF660002070795
:1014B00007060066FFFFFFFFFF1F00060707070282
:1014C000001FFFFFFFFFFF26040607070706002691
:1014D000FFFFFFFFFF1F000607070706041FFFFFB0
:1014E000FFFFFF660006070707020066FFFFFFFF1A
:1014F000FF1F00020707070600FFFFFFFFFFFFE6D1
:1015000004060707070702E6FFFFFFFFFFFF0207CA
:101510000707070604E2FFFFFFFFFF3A0006070781
:101520000702003AFFFFFFFFFFE20002070707067E
:101530000056FEFEFFFFFFDE0000050F1F0F1DDE41
:10154000FFFFFFFEFE561D0F1F0F0500000A0D00D6
:10155000004094BCB6FAD68C40000000000005099B
:1015600005080000FE4094BCB6FAD68C4010070077
:10157000000005090508000E0D000018ACF46C7899
:10158000A80000000000000008060B070101000091
:1015900000000000000000000080C0C0A070E0401B
:1015A00000000000000A0A0703050305000100000F
:1015B000000080008000808080008040C0800000AB
:1015C00000040200030709070F050E0300070B00C4
:1015D0000ADEFB9D6B0600040204060000066B9DFC
:1015E000FBDE0A00000006040204004A1EDBFDEBDD
:1015F0002640000002040600004026EBFDDB1E4AE8
:10160000000006040200000A1EDBFDEB660000007D
:1016100002000600000066EBFDDB1E0A000006006B
:101620000200000A1EDBFDAB2600000402000600DB
:10163000000026ABFDDB1E0A000006000204000AC3
:101640001EDBFDEB6600000006000200000066EBFA
:10165000FDDB1E0A000002000600004A1EDBFDEB57
:101660002640000402000202004026EBFDDB1E4A79
:10167000000202000204004022EBFBEB22100000FB
:1016800006000200001022EBFBEB224000000200EB
:1016900006000054BCB6FAD60C0000000509050887
:1016A000000CD6FAB6BC5400080509050000001469
:1016B00014000000C03804C2796551516579C20434
:1016C00038C000000038C40213E4E9A2D735E5E5CC
:1016D00035D7A2E9E41302C438000C050A08090D45
:1016E0000A010101010A0D09080A050C00000000A9
:1016F00000C03844DAE5F9C5338A74887080000088
:101700000000000043249B0706973379381010002F
:1017100080010608F000060D0F07000809060D0FEE
:10172000070008060908000E010000008070887498
:101730008A33C5F9E5DA4438C000000000F0080635
:1017400001800010103879339706079B244300006E
:1017500000010E000809060800070F0D0609080021
:10176000070F0D0600C03008087CF4C21D2B416B2A
:10177000412B9EC47C080830C00738C012C4E8E280
:10178000F7F56565F5F7E2E8C412C03807000C0507
:101790000A08090D0B010101010B0D09080A050CCE
:1017A00000000000C0380402D9A511B115A1C2047F
:1017B00038C000000078848203CFCFECF1E2646689
:1017C000E4F2E9CCC703828478000C050A08090D0D
:1017D0000B010101010B0D09080A050C00000000B6
:1017E000C03804C2796551516579C20438C000001F
:1017F0000070888403C4D982385482D682543881D8
:10180000C403848870000C050A08090D0B0200004F
:10181000020A0D09080A050C00000000C03804C2C5
:10182000796551516579C20438C000000038C4029E
:1018300013E4E9229745256525478229E41302C46C
:1018400038000C050A0809080305080D08050308F7
:10185000080A050C0000000000C020109010C8A469
:101860002272CAAA4A02E408F00018648847307954
:10187000FEFC7132254A2C09877108040300000020
:101880000000020504080A05010101010000000032
:1018900000E8182090C8C8C424844830A020204004
:1018A0004040800000C38142BDDB5ABD66007EC35C
:1018B0007E81FF665A4224817E070804090B0B0BC8
:1018C0000C090A0C050404020202010000D0F8F819
:1018D000F0F8F8F8FCFCFCF8F0E0E0E0C0C0C080F4
:1018E00000000087CF87FFFFFFFFFFFFFFFFFFFF25
:1018F000FFFFFFFFFFFFFFFEFC0F1F3F1F3F3F3FAC
:101900003F3F3F3F3F1F1F1F0F0F0F0703010016F1
:101910001600D030402090908848089060404040A9
:1019200080808000000000008702847BB7B57BCCFC
:1019300001FC86FD02FECCB4844902FC00000F11BC
:101940000813171617181214190A090904040402B7
:10195000010000000000C0E0F0F8F8F8FCFEFFFF16
:10196000FFFFFFFFFEFCF8F0187CFEFFFF7FFFFF8C
:10197000FFFFFFFFFFFFFFFFFF7F0F0703000000D8
:101980000102070F0F1F1F0F0703030301000000D1
:101990000000151500000000C020109010C8A422FF
:1019A00072CAAA4A02E408F0000018648847307935
:1019B000FEFC7132254A2C098771080403000000DF
:1019C000000000020504080A0501010101000000F1
:1019D00000000000000080F0F8FCFEFFFFFFFFFFAA
:1019E000FFFEFCF8F08000000070F8FCFFFFFFFF36
:1019F000FFFFFFFFFFFFFFFFFFFFFFFFFCF870008F
:101A0000193F1F3F3F3F3F3F170707173F3F3F3FEC
:101A10003F1F3F190016160000000080700884F276
:101A2000CAA2A2CAF2840870800000000000708878
:101A30000427C8D245AE6ACACA6AAE45D2C82704CE
:101A40008870000000190A1411131B150203030209
:101A5000151B1311140A190000387CFEFFFFFFFE4E
:101A60007C38000000010101000000090900385421
:101A700082D6825438000000000000000000000000
:101A8000384CC2928664380000000000000000005C
:101A9000000038648692C24C38000000000000004C
:101AA000000000B8014B00FF7F0200008000000131
:101AB000000001000001000001FF0304FF0304FE19
:101AC0000506FE0506FF0708FF0708070D06070DB8
:101AD000060B0E040B0E040D10010E100112120362
:101AE0001312031514051514051616071718070AFF
:101AF00000090000020000020000020000020003D2
:101B000002000602000902000C02000F020012028D
:101B100000140200000900000000000000000000A6
:101B20000000010303010303010505010505010789
:101B300007010707010009DC00B400DC005A00DCE3
:101B4000005A00DC00B400DC00B4001501B400DC75
:101B500000B4001501B400DC00B4000080000204F1
:101B60000608090A0A0B0B0C0C0C0D0D0D0D0D0DC2
:101B70000D0D0D0D0D0D0C0C0C0B0B0A09080604B8
:101B800002007F4A027D4A027B4A02794A02774A72
:101B900002754A02734A02714A026F4A026D490293
:101BA0006B4902694902674902654900634900615E
:101BB00049005F49005D49005B49005949005748A9
:101BC000005548025348025148024F48024D48020E
:101BD0004B480249480247480245480143470141F2
:101BE00047013F47013D47013B470139470137471F
:101BF000013547023347023147022F46022D460284
:101C00002B4602294602274602254600234600218C
:101C100046001F46001D46001B450019450017459C
:101C2000001545021345021145020F45020D4502FC
:101C30000B45020945020744020544010344010122
:101C40004401FF4401FD4401FB4401F94401F74410
:101C500001F54401F34302F14302EF4302ED430275
:101C6000EB430200000288011400AF001400008062
:101C70002C003200210032003700320000801003B7
:101C80003200930232000B023200700332005D0119
:101C9000320026013200EE0132000080B8014B0014
:101CA000EE014B002A024B00100396006E029600D4
:101CB0000080E402F20100009000E4022200000033
:101CC0004800E402220000004800E402B1000000E5
:101CD0006C00E402690000002400E40246000000F9
:101CE00048003F03690000002400A40369000000CD
:101CF0002400DC030A040000FB00DC036900000090
:101D000024005504460000004800DD0446000000A1
:101D1000480075055D0200002400750522000000E2
:101D200048007505220000004800750522000000EB
:101D3000B3005504B1000000240075054600000002
:101D40004800C8057500000018007D066900000005
:101D50002400C80569060080AF0014008801140043
:101D6000008010033200930232000B023200700335
:101D700032005D01320026013200EE013200C40063
:101D80003200A500320083003200DC003200570030
:101D90003200490032008000320080003200000032
:101DA0001400800032000000140080003200008027
:101DB000181E1000190100050F0C18042418053C0A
:101DC00018060943001342001D4100274000313F1F
:101DD000003B3E00453D00092F03152F01212F0137
:101DE0002D2F01392F01452F01174B01234B01578F
:101DF00050015F50016B50017750016349016F49F9
:101E0000017B49016B500E573F01633F016F3F015A
:101E10007B3F01FB6C01166C01226C012E6C0132C0
:101E20006C014F6C01005C000A5D00145E001E5FD7
:101E3000002860003261003C62004663005064008C
:101E40005A65007170027D70020A85001484001EBC
:101E500083002882003281003C8000467F00507E53
:101E6000005A7D00647C00094A035B6A03FC2F0171
:101E70000024070044891444882845883C4688503B
:101E800047886448887849885B0A0A55000B007ABD
:101E90000C007A4D000000FFFFFFFFFFFFFFFFFF78
:101EA000FFFFFFFFFFFFFFFFFFFF0000000000003C
:101EB000000000F0F8F0F0F0F0F0F8F01402030386
:101EC00000030303000303030003030300030303EE
:101ED00000030707000707070007070700070707B2
:101EE000000707070007FFFFFFFCFCFCFCFCFFFFEF
:101EF000FFFFFFFFFFFFFFFFFFFFFFFF07070701D8
:101F00000101010107070725200000000000000073
:101F100000000000000000000000000000000000C1
:101F200000000000000000000000000000000000B1
:101F3000000000008040200C1A1ECCC0828A36E4CB
:101F40008444A84818D09010202020404040808031
:101F50008000003048482502040000000000000016
:101F60000101030307070F0C1C1838337E78F4CAED
:101F7000C582810E7CE0010100000000000000002D
:101F80000000000000000000000000000000000051
:101F900000000000000101030307070F0C00000010
:101FA0000000000000000000000000000000000031
:101FB0000000000000000000000000000000000021
:101FC0000000000000000000000000CC1A1ECCC081
:101FD000828A36E48444A84818D0901020202040FB
:101FE00040408080800000000000804042340813A0
:101FF000200000000101030307070F0C1C183833F1
:102000007E78F4CAC582810E7CE0010100000001E7
:1020100002020100000000000000000000000000BB
:102020000000000000000000000101030307070F8B
:102030000C00000000000000000000000000000094
:102040000000000000000000000000000000000090
:102050000000000000000000000000000000000C74
:10206000DA1ECCC0828A36E48444A84818D0901086
:1020700020202040404080808000000000000000C0
:1020800000000000887B08000101030307070F0C14
:102090001C1838337E78F4CAC582810E7CE00101B9
:1020A000000000000000000000010202010000002A
:1020B000000000000000000000000000000101031B
:1020C0000307070F0C0000000000000000000000E4
:1020D0000000000000000000000000000000000000
:1020E00000000000000000000000000000000000F0
:1020F0000000000C1ADE0CC0828A36E48444A84832
:1021000018D09010202020404040808080000000A7
:102110000000000000000000000020139869058105
:1021200007070F0C1C1838337E78F4CAC582810E5D
:102130007CE0010100000000000000000000000041
:102140000001020201000000000000000000000089
:10215000000101030307070F0C000000000000004E
:10216000000000000000000000000000000000006F
:10217000000000000000000000000000000000005F
:10218000000000000000000C1A1E4CC0028A36A499
:102190000444A84818D0901020202040404080805F
:1021A00080000000000000000000000000000000AF
:1021B000080402056893876C0C1838337E78F4CADB
:1021C000C582810E7CE001010000000000000000DB
:1021D00000000000000000000000000000000000FF
:1021E00000000000000101030307070F0C25180081
:1021F0000000008040C08020A0A0202020A020D08F
:10220000D09010101010109050906868C88808087E
:102210000808080800000000017B0301080C0D0FEE
:102220000E0D0E1D1818191B1E1C1A1D1A19181038
:1022300010303133363C38343A00000000314F4121
:10224000200000000000000000000000000000006E
:1022500000000000000000000000000000001C283A
:10226000000000000000000000000000000000006E
:102270000000008080C0C060603030180000008026
:1022800080C0C060603030B8188C6CE6C68383E1D3
:1022900019E4168C8C98587418B43C190120222625
:1022A0001C1816090E0904040403030301010100AC
:1022B00000000000887B0800000000000000000013
:1022C000000000000000000000000000000000000E
:1022D00001020201000000000000000000000000F8
:1022E0000000000000000000000000003F1000009F
:1022F0000000000000000000F018D85818D8D818C6
:10230000D8D818D8D818F87880C0C0C0C0C0C0C00D
:10231000C0C0C0C0FE03DBDB03DBCB03DBDB03DBC6
:102320005B03FFFF00000000000000000020000031
:10233000202000202020203F0036160036360036B0
:1023400032003636003F0036160036360036320090
:102350003636003F00363200363600361600363646
:10236000003F3F20202000202020002013080000F4
:102370007C54440078147800485424000C700C00FD
:102380000000007C107C00781478007C1468007CCD
:10239000443800000910000000000000000000F0B8
:1023A00008D0D010101008F00C14004210000044A7
:1023B00010004008010020D089A8A8A8A988B08CE6
:1023C000D3200002050B0F0A0A0A0A050200008842
:1023D0002000000842000044100220D088A8A8A9CC
:1023E000A888B08CD3200002050B0F0A0A0A0A0540
:1023F000020000820010440000104200080020D0BB
:1024000088A9A8A8A889B08CD3200002050B0F0AC0
:102410000A0A0A05020000421000004410000008E9
:102420004100408091285060115860B18040000107
:1024300003070F0F0F0F070301000088200000089B
:10244000420000441002408090285061105860B053
:102450008140000103070F0F0F0F07030100004128
:102460000800001044000010420040809128506194
:10247000105860B18040000103070F0F0F0F0703D2
:10248000010000000000008040800000000000808B
:1024900040582E2F2F96954A800003040A0A0D0DEE
:1024A0000D0E0E0B05030910000048B0CCB0420021
:1024B00000F008DFDB151B1F08F0000080E862C099
:1024C000D00000F008DFD41B141F08F0000080E8E3
:1024D00072C0D00000F008DFD41B141F08F0000009
:1024E00002B058A4F00000F008DFDF151E1F08F04E
:1024F000091B0000805C7B5C0000000609102020A6
:102500002010080000000000000000000000000093
:102510000000000000000000805C7B5C0000000602
:10252000C91020202010080000FF0000000000005B
:10253000000401000000000000000000805C7B5CE3
:1025400000000006C910A0202010080000FF00FFB6
:102550000000000000040104010000000000000071
:10256000805C7B5C00000006C910A020A010080061
:1025700000FF00FF00FF000000040104010401004F
:1025800000000000805C7B5C00000006C910A020F9
:10259000A010C80000FF00FF00FF00FF00040104BE
:1025A0000104010401001A20000000000000008066
:1025B0004018B4BC180008D0B02040808000000053
:1025C00000006090904A0408010000000003070C1E
:1025D0003973E898141415D3D6140C1800000000B1
:1025E0000000000000000000000000000103071CC4
:1025F00038F3CD940A0A000000000000000000003B
:1026000000000000000000000000000001030F1E99
:102610000000000000000000009834BC180008D042
:10262000B020408080000000000000000000808496
:10263000681026010003070C3973E898141415D3A9
:10264000D6140C180000000304040200000000006F
:10265000000000000103071C38F3CD940A0A0000B3
:10266000000000000000000000000000000000006A
:102670000000000001030F1E000000000000000029
:102680000018B4BC180008D0B020408080000000C2
:10269000000000000000000000000040DE43070CC6
:1026A0003973E898141415D3D6140C1800000000E0
:1026B00000000000000C1310080000000103071CBC
:1026C00038F3CD940A0A000000000000000000006A
:1026D00000000000000000000000000001030F1EC9
:1026E00014020100000001000000010000000100D0
:1026F00000000100000014030200000002000000BE
:102700000200000002000000020000000B0BF8387D
:1027100078E8D0A000A0100C0C07040404050707FB
:1027200007000000F83878E0C8A4438300000007E1
:10273000040404050707070000000B1300FE4848C7
:102740004848484848FE0000FF9292929292929226
:10275000FF0000030000000000000003001910014A
:10276000010705050703030303030303030303032F
:102770000303070505070404000000000000000033
:102780000000000000000000000000000000000049
:1027900000040407050507030303030303030303FE
:1027A0000303030307050507010100000000000003
:1027B0000000000000000000000000000000000019
:1027C00000000001010705050703030303030303DA
:1027D00003030303030307050507010100000000CD
:1027E00000000000000000000000000000000000E9
:1027F000000000000001010F0B0A0E060606040C83
:102800000C0C081818181870505070404000000048
:1028100000000000000000000000000000000000B8
:102820000000000000000000404070505070181878
:102830001818080C0C0C040606060E0A0B0F0101F2
:102840000000000000000000000000000000000088
:1028500000000000000000000001070B0A0E060443
:102860000C0C08181810303020E06040C000000048
:102870000000000000000000000000000000000058
:102880000000000101010101000000000000000043
:10289000C04060E0203030101818080C0C04060E00
:1028A0000A0B070100000001010101010000000006
:1028B0000000000000000000000000000019362C9D
:1028C000183060C080000000000000000000000020
:1028D00000000000000000000000000000010306EE
:1028E0006CD8B06080000000000000000000000014
:1028F00000000000000000000000000000000000D8
:1029000080C06030182C3619000000000000000064
:1029100000008060B0D86C060301000000000000D9
:10292000000D08252D39312931252D393129312145
:102930000C08627A7A62627A7A62627A7A620B0848
:10294000878F9DB7E7C7A5D7AF978D0208D4D2056B
:10295000087F7F3E1C084120FE0105F1F1F111D1F5
:10296000B1D111F151515151515151515151515117
:1029700051510000FF00007F7F09090F06007F7F93
:1029800019396F46007F7F4949414100266F494907
:102990007B3200266F49497B32FF0000FFFFFFFEBC
:1029A000FFFEFF0279CD95A5CD790111111101F935
:1029B000F901010000FF00007F7F09090F06007F79
:1029C0007F40404040007C7E0B0B7E7C00070F78F0
:1029D000780F0700000000000000FF00001F3F3FCD
:1029E00033333333333E36363E363E363E36363E6E
:1029F00036363E360000FF00003E7F41417F3E00FC
:102A00007F7F0E1C7F7F00000000000000000000A0
:102A100000000000000000000000003F4050404067
:102A200040784641415959414141415959414141FB
:102A3000414141414100007F000001017F7F0101D0
:102A4000007C7E0B0B7E7C007F7F09090F06007FD8
:102A50007F49494141000000000000005700680123
:102A60003E006801570068013E006801AF00B400F5
:102A70009C00B400AF00B4009C00B400000019003A
:102A80009C005A0000005A009C005A0000005A00A6
:102A90009C005A0000005A009C005A0000005A0096
:102AA000C4006801B9006801C4006801A50068019C
:102AB000AF005A00A5005A00AF005A00A5005A0006
:102AC000AF005A00A5005A00AF005A00A5005A00F6
:102AD000AF00EE020080FFFFFFFFFFFFFFFFFFFFE1
:102AE000FFFFFFFFFFFFFFFFFFFFFFFFFFFFFFFFF6
:102AF000FFFFFFFFFFFFFFFFFFFFFFFFFFFFFFFFE6
:102B0000FFFFFFFFFFFFFFFFFFFFFFFFFFFFFFFFD5
:102B1000FFFFFFFFFFFFFFFFFFFFFFFFFFFFFFFFC5
:102B2000FFFFFFFFFFFFFFFFFFFFFFFFFFFFFFFFB5
:102B3000FFFFFFFFFFFFFFFFFFFFFFFFFFFFFFFFA5
:102B4000FFFFFFFFFFFFFFFFFFFFFFFFFFFFFFFF95
:102B5000FFFFFFFFFFFFFFFFFFFFFFFFFFFF44102F
:102B6000000000000000BC7EC7EBEDEBC77EBC00A0
:102B7000003C2C00381438000824100004380400ED
:102B80000000000000BC7EC1D5D5D5CB7EBC0000C6
:102B90003C103C00381438003C1428003C24180039
:102BA000000000000000000000000001020202021C
:102BB0000201000000000000000000000000000012
:102BC00000000000000000000000010202020202FA
:102BD00001000000000000000000000000000000F4
:102BE0000000000000000000387CFEFFFFFFFE7CBC
:102BF000380000000101010000000909003854827A
:102C0000D6825438000000000000000000000038A8
:102C10004CC29286643800000000000000000000F2
:102C20000038648692C24C380000000000000000AA
:102C300000000D08252D39312931252D3931293153
:102C400021622BFC02FDFDFDFDFDFDFDFDFDFD02F4
:102C5000FDFDFDFDFDFDFDFDFDFD027C90E8F4FAAE
:102C6000FDFDFDFDFDFDFDFDFDFDFAF4E890FC021E
:102C7000FDFDFDFDFDFDFDFDFDF3CC02FDFDFDFDBA
:102C8000FDFDFDFDFDFDFD02DCE8F4FAFDFDFDFDB1
:102C9000FDFDFDFDFDFDFAF4E8D020C000000000C0
:102CA00000000000000001FE00FFBF7F7F3FBFBFAC
:102CB000BC7E7F7FBF7FB7CB35C20202FF00FFBF64
:102CC0007FBF7FBFFF01FE0001FF7FBF7FBF7FFF90
:102CD00000FFFE00FFBF7FBF7FBFFF7FFFBF7CB055
:102CE0007FBF7FBF7FBFFF00FE00FFBF7FBF7FBFF3
:102CF000FF00FE0EECAB6BAB6BAB6BEB0CF30000B1
:102D000000000000000000F008F7B0DFAAD0800348
:102D1000354E7D6F15FAAFD5AAD7AED9B6F40FF000
:102D20008F7AD5AAD5AADFB8D7B4D8AFD5AAD5EAB5
:102D30007D8FF00FF7B0DFAAD5AAD5AADFB0F107D3
:102D40009D7AD5AAD5AAD5AAFF00FF40BF6AD5AA09
:102D5000D5AADFB0D7B4D3BED56A350A959F809F78
:102D60008080000000000000003B78EABA3A3A2A6E
:102D7000BA78B86B3A79EAB83A3A2ABA7ABA6A3A79
:102D800078EBB8393A28BA7ABA6A3A7AEABA3A3A69
:102D900028BA79B86B387AEABA3A3A2ABA7ABA6A69
:102DA0003A78EBBA383A2ABA7ABA6A387BE8B8394C
:102DB0003A28BA7ABA6A3A3A0A00E01C8261BCB28E
:102DC000A8A8B2BC61821CE000000004040405074E
:102DD00006050605040404040405070605060504A3
:102DE0000404040405070605060504040404040598
:102DF0000706050605040404040405070605060580
:102E00000404040404050706050605040404040478
:102E10000507060506050400001C62810972F4D14D
:102E20006B9AF2F29A6BD1F4720981621C00000075
:102E30000000000000000000000000000000000092
:102E40000000000000000000000000000000000082
:102E50000000000000000000000000000000000072
:102E60000000000000000000000000000000000062
:102E70000000000000000000000000000602050441
:102E800004060500000000050604040502060038DB
:102E90007CFEFFFFFFFE7C38000000010101000006
:102EA00000090900385482D682543800000000001E
:102EB000000000000000384CC29286643800000018
:102EC000000000000000000038648692C24C380008
:102ED00000000000000000000003F70403F80403F2
:102EE000F90403FA0403FB0403FC0403FD0403FEDA
:102EF0000403FF04030004030102050102070102A9
:102F00000901020B01020D02020F0202110202135B
:102F100002021502021703021903021B03021D031A
:102F2000021F0302210402230402250402270402D3
:102F30002904022B05022D05022F0502310502335B
:102F400005023506023706023906023B06023D0637
:102F5000023F0702410702430702450702470702F3
:102F60004908024B08024D08024F0802510802535B
:102F700009025509025709025909025B09025D0A53
:102F8000025F0A02610A02630A02650A02670B0213
:102F9000690B026B0B026D0B026F0B02710C02735B
:102FA0000D04730F04731104731304731504731762
:102FB00004731904731B04731D04731F0473210429
:102FC0007323047123016F23016D23016B240169B5
:102FD00024016724016524016324016125015F2523
:102FE000015D25015B250159250157260155260163
:102FF0005326015126014F26014D27014B27014938
:1030000027014727014527014328014128013F287F
:10301000013D28013B2801392901372901352901C2
:103020003329013129012F2A012D2A012B2A0129B7
:103030002A01272A01252B01232B01212B011F2BDC
:10304000011D2B011B2C01192C01172C01152C0122
:10305000132C01112D010F2D010D2D010B2D010937
:103060002D01072E01052F0105310105330105351D
:1030700004053704053904053B04053D04053F04F8
:10308000054104008A3011241FBECFEFDAE0DEBF15
:10309000CDBF11E0A0E0B1E0E2E0FAE602C00590A9
:1030A0000D92AE33B107D9F726E0AEE3B1E001C02F
:1030B0001D92AE3AB207E1F718E1C3E4D8E104C0CB
:1030C0002197FE010E94F934C234D107C9F70E944A
:1030D00052310C94FF340C94000090E121E061FD2A
:1030E00024E060FD220F62FD2295687F969FD0014B
:1030F0001124A80FA255BD4F8C91822B8C9308955B
:10310000A7E9B2E02FB7F8947D918D919C9166B5B7
:103110002FBFA89B05C06F3F18F47F5F8F4F9F4F55
:1031200022E0660F771F881F991F2A95D1F708950F
:103130006F927F928F929F92AF92BF92CF92DF92C7
:10314000EF92FF920F931F93CF93DF934C01DB011C
:1031500058017C2D4115510509F4A0C0FA01649174
:10316000319684914E5F5F4FC62FD0E0211102C08F
:10317000EE2009F1E1E0F0E0982F977011F4F0E013
:10318000E0E0082F0695069506950E0F1F2F111DDE
:103190000C9FF0010D9FF00D1C9FF00D112473305A
:1031A00009F08BC0EE0FFF1F2E9F80012F9F100D87
:1031B0001124400F511F84010C0F1D1F1016110602
:1031C0000CF06CC0F0E88F1691040CF067C09D0104
:1031D000280F311D121613060CF060C0A034B10583
:1031E0000CF05CC04115510509F458C03A2F3770F6
:1031F000FD01B7FD379693E0F595E7959A95E1F7D0
:103200002E2FB7FF04C0332311F02FEF2E0FEE2720
:10321000FF27E819F90997FC02C0F0E0E0E090E828
:103220009819003811050CF4962F9E1BA22F022E20
:10323000000CBB0B1A2F10952F3F0CF010E0DD2473
:10324000D394082F077009F4D12C8695869586951E
:10325000D80EAD0DB11D19971CF0A8E0DA2ED21AC8
:10326000D11A210F00E82003D0011124A80DB91DA7
:10327000AE0FBF1F619FE00DF11D11244E0F5F1FA8
:10328000E32E032E000CFF08733009F424C108F567
:10329000713009F4D6C0723009F484C0DF91CF9147
:1032A0001F910F91FF90EF90DF90CF90BF90AF9064
:1032B0009F908F907F906F900895A114B10409F4AE
:1032C00073CFEE9E8001EF9E100D1124A00EB11E53
:1032D0006BCF7A3FB1F10D2D020F7B3FF9F620172E
:1032E000E9F2BD0162557D4FD12CC12CC91608F001
:1032F000A2C0FA01EC0DFD1DE491F0E04F010E2C8F
:1033000002C0880C991C0A94E2F727FD06C0FB0155
:103310008081182D109581238083332361F027301D
:1033200054F45B01F0E8AF0EB11C192D1095F501B6
:10333000808181238083FFEFCF1ADF0A6F5F7F4F89
:10334000D5CF0D2D020F201709F4A8CFBD0162556E
:103350007D4FD12CC12CC91608F067C0FA01EC0DC5
:10336000FD1DE491F0E04F010E2C02C0880C991C69
:103370000A94E2F727FD04C0FB018081882980833D
:10338000332351F0273044F45B01F0E8AF0EB11C59
:10339000F501808189298083FFEFCF1ADF0A6F5FF3
:1033A0007F4FD9CF6FEF70E0032E02C0660F771FFB
:1033B0000A94E2F760957095972E8D2C820E281551
:1033C00009F46CCF8D0102551D4FD12CC12CC916AB
:1033D00030F5FA01EC0DFD1DE491F0E03F010E2CFB
:1033E00002C0660C771C0A94E2F727FD05C0F801BD
:1033F0008081862386298083332359F027304CF43B
:103400005801F0E8AF0EB11CF501808189218729B0
:103410008083FFEFCF1ADF0A0F5F1F4FD8CF2F5FD8
:103420004C0F5D1FA058BF4FCACF2F5F4C0F5D1FC1
:10343000A058BF4F88CF2F5F4C0F5D1FA058BF4FC4
:103440004ECF85010E0F1F1F8D2D820F281709F4F7
:1034500025CFBD0162557D4FD12CC12CC91698F5E1
:10346000F801EC0DFD1DA490B12C0E2C02C0AA0C8D
:10347000BB1C0A94E2F7A094B094FA01EC0DFD1D78
:103480008490912C0E2C02C0880C991C0A94E2F7AF
:1034900027FD08C0FB017080E72DEA217E2E7828E9
:1034A000FB017082332349F027303CF4FB01E058E4
:1034B000FF4FA080BA20B928B082FFEFCF1ADF0AF1
:1034C0006F5F7F4FCBCF2F5F4C0F5D1F0C0F1D1F0A
:1034D000A058BF4FBBCFE92EF12CE40FF51FA2552A
:1034E000BD4F60E870E06E197F09CE19DF09AE01AB
:1034F000440F551FC1E0D0E07E01032E01C0EE0C49
:103500000A94EAF7192F0D2D892E932ECF93DF936E
:10351000ED01EF96EF962296A590C590992059F06F
:10352000AE9C5001CE9C600127302CF4F880D094E2
:10353000FD20FB28F99222233AF0FC90C094FC2055
:10354000FA28FD920C94A51A11961A9529F70A9556
:1035500051F0182D23951124E40FF11DA60FB11D74
:10356000C60FD11DD9CFDF91CF91112497CECF9225
:10357000EF920F931F933AEFC32EE12C10E000E07F
:103580000E9498181F910F91EF90CF900895CF92BD
:10359000EF920F931F9332E0C32EE12C10E000E076
:1035A0000E9498181F910F91EF90CF900895CF929D
:1035B000EF920F931F93F901202FCC24C3948F0116
:1035C0000E9498181F910F91EF90CF900895EF925D
:1035D0000F931F93CF93DF93EA0123E0629FB00123
:1035E0001124FB01E752F14D1491FB01E652F14D1C
:1035F0002491FB01E552F14DE491DC0115968D918A
:103600009C9165E070E00E94D134892BA1F4E130F7
:1036100059F0E23081F48881823020F48F5F888312
:1036200008810CC080E0FBCF8881882311F0815095
:10363000F6CF82E0F4CF00E0E43091F7622F220F62
:10364000770BE12C2FE83EE241EA5EE2812F90E029
:103650000E94D71ADF91CF911F910F91EF9008959B
:10366000BC0190E080E0AB01FC010E948018415059
:103670005109E109F10928F068517C4F8F4F9F4FA4
:10368000F6CFAB01FC010E948018641775078E0706
:103690009F07C8F308958FB18095807F669B8860EF
:1036A0001C9B846008958091900208950895EF9284
:1036B0000F931F93CF93DF93EC0120E041E45CE292
:1036C00066E070E084E190E00E94C71A0BE010E031
:1036D00020E042E35CE262E370E0C8010E94B71AB6
:1036E000045F1F4F0737110599F79A89E12C0B8961
:1036F00028EE3BE24AEF5BE269E270E0E3E3F0E0F0
:10370000DF01A91BB109CD010E94D71A8A8990E077
:103710000C8928EE3BE24AEF5BE269E270E0C39677
:103720000E94D71A8989823859F400E026ED3AE2DE
:103730004EE55BE26EE270E086E190E00E94D71A0F
:10374000DF91CF911F910F91EF900895CF93DF9369
:10375000EB0120E046E559E261E170E080E290E0B3
:103760000E94C71A8D819E8160E370E00E94D1346F
:10377000883170F4C1E18C3008F0CEE120E04FE4F4
:1037800059E269E170E08BE590E00E94C71A04C03D
:10379000CFE1843208F0C0E26C2F70E084E390E067
:1037A0000E946D18C0FD0BC020E04BE459E26CE1B3
:1037B00070E08DE290E0DF91CF910C94C71ADF9119
:1037C000CF91089583E59BE190938D0280938C02C5
:1037D00010928F0210928E0281E080938F020895E2
:1037E000FC01DC01A256BF4F1C9211971C9213964C
:1037F00081E08C9311971C92139682E08C93119721
:103800001C92118A128A138A8DE0848B138E158A7A
:10381000E656FF4F84E080830895FC01E758FF4F90
:1038200021E02783BA961082319628EC20833696C1
:1038300010827A97138210820480F581E02D82E055
:10384000828384E18083FB0180898150808B08958D
:10385000FC018581843019F0883029F00895838136
:1038600081508383089583818F5FFBCF2F923F9296
:103870004F925F926F927F928F929F92AF92BF9280
:10388000CF92DF92EF92FF920F931F93CF93DF932C
:10389000CDB7DEB728970FB6F894DEBF0FBECDBF09
:1038A0005C018B01FC01838D650181111DC1FCE16F
:1038B000CF0ED11CF80145805680EAE08E2E912C67
:1038C000F3E0EF2EF12C20E046E150E1B401C70116
:1038D0000E94B71AFAE0EF0EF11C2FEF821A920A3B
:1038E00031E7E316F10479F766E3862E912C7FE049
:1038F000E72EF12C20E046E150E1B401C7010E941F
:10390000B71A8AE0E80EF11C91E0891A9108EDE7F8
:10391000EE16F10479F7A5014C5E5F4FF501618960
:10392000C8010E94E71AA5014B5E5F4FF50162894D
:10393000C8010E94E71AA5014A5E5F4FF50163893D
:10394000C8010E94E71AF8018581968165E070E060
:103950000E94D134892BB1F4F50181898D3808F0AA
:10396000C7C08F5FF501818B82898D3808F0C2C096
:103970008F5FF501828B83898D3808F0BDC08F5F22
:10398000F501838BE12C00E024E43DE04CEA5EE0AD
:1039900062E170E08DE190E00E94D71A28E33BE0FD
:1039A0004DE35CE063E070E086E190E00E94D71AAE
:1039B000760108E110E09E012F5F3F4F19013701AA
:1039C00032E0630E711C54E2852E912CF30121919B
:1039D0003F012F3309F492C0205442EA5AE0B80163
:1039E000C4010E94C71AF6E08F0E911C26E38216CE
:1039F000910461F73E0137E0630E711C41E4842EAF
:103A0000912C78866F82F10126E011922A95E9F7D0
:103A1000F70180819181F1016AE070E00E94D13468
:103A20008193CB012F8138852E173F07A9F7F3012A
:103A300022913F01255E42EA5AE0B801C4010E948A
:103A4000C71AF5E08F0E911C2FE582169104D9F666
:103A5000075F1F4F36E0E30EF11C0333110509F039
:103A6000AECFF50107890F3F09F470C0C20168E2CB
:103A700070E00E94D134853108F468C086E0089F68
:103A800010011124F2E02F0E311C29E0029F800169
:103A90001124280137E1430E511CF501608C689E0A
:103AA000300111247301F3E2EF0EF11C29E2620EE2
:103AB000711C015E1F4FE614F70431F14201C80189
:103AC0000134110514F080E490E088169906C4F4DE
:103AD00030E8E316F10424F4B401C7010E946D1824
:103AE0008FEF881A980AEBCF2EE2C20ED11CE2CEDD
:103AF00080E038CF80E03DCF80E042CF20E06DCF46
:103B00009FEFE91AF90AD7CFF501808DC20CD31CBB
:103B1000F601E80FF11D20812F3309F450C0205425
:103B2000F5016789F9E06F9FB0011124685E7F4F4E
:103B300036E0839FC00111243BEFC32EE12C10E03F
:103B400000E042EA5AE084960E949818F5018789BD
:103B50008F3F79F4828D81110CC0E12C00E02CE1C3
:103B60003AE04EE55AE065E370E080E390E00E94C1
:103B7000D71AE12CF501038D2EE739E042EB59E02D
:103B80006BE170E082E090E00E94D71A28960FB6B1
:103B9000F894DEBF0FBECDBFDF91CF911F910F9183
:103BA000FF90EF90DF90CF90BF90AF909F908F905D
:103BB0007F906F905F904F903F902F90089520E0FE
:103BC000AFCFDC0185E0869F9001879F300D1124E7
:103BD000F901E35BFC4F5491F901E25BFC4F449126
:103BE000F901E15BFC4F9491F901E05BFC4F84919A
:103BF0002F5A3C4FF90124915C9311964C931197E5
:103C000012969C93129713968C93139714962C9359
:103C10000895CF93DF93EC01198218821A8270E025
:103C200060E00C960E94E11D1A821F821886198698
:103C30008FEF8C8388E08E83DF91CF910895FC0114
:103C40008181813071F020F0823099F080E0089518
:103C5000E08183E0E89FF0011124E85EF44E849156
:103C60000895E08183E0E89FF0011124EC50F54EC7
:103C7000F6CFE08183E0E89FF0011124E155F54E95
:103C8000EECFFC018181813071F020F0823099F01B
:103C900080E00895E08183E0E89FF0011124E95E6F
:103CA000F44E84910895E08183E0E89FF0011124AF
:103CB000ED50F54EF6CFE08183E0E89FF00111244E
:103CC000E255F54EEECFFC018181813071F020F09C
:103CD000823099F080E00895E08183E0E89FF00170
:103CE0001124EA5EF44E84910895E08183E0E89F18
:103CF000F0011124EE50F54EF6CFE08183E0E89F0D
:103D0000F0011124E355F54EEECF2F923F924F92E2
:103D10005F926F927F928F929F92AF92BF92CF925B
:103D2000DF92EF92FF920F931F93CF93DF93CDB764
:103D3000DEB72D970FB6F894DEBF0FBECDBF7B83E5
:103D40006A834983FC01E758FF4F468420EBC22E6B
:103D50002DE1D22E34E9232E3EE1332E512C5C018D
:103D600027E9A20EB11CDC01AA56BF4FBD83AC836C
:103D7000B196FF83EE839C0126573F4F39872887F2
:103D80001697BB87AA874C01B1EA8B0E911C3C01A8
:103D9000EFE96E0E711C2D5E3F4F3D872C87F601BB
:103DA000F4903196E49031968491E491F981F11187
:103DB00022C0E6FF25C0F3E0CF0ED11C2C143D0439
:103DC00071F780E02D960FB6F894DEBF0FBECDBF21
:103DD000DF91CF911F910F91FF90EF90DF90CF90E7
:103DE000BF90AF909F908F907F906F905F904F901B
:103DF0003F902F90089529812034E9F6E6FFDBCF2C
:103E0000AA81BB8152960C91013011F0E7FDD3CF0E
:103E10008F71813180F6E82FF0E0EF5EF04E0C9468
:103E2000F934BB1FCC1FC61FD81F221F311F4E1FC6
:103E3000581FC01FDE1F601F831F8B1FA61FB61FCA
:103E4000931FD21F8C859D850E94631E082F8C8531
:103E50009D850E94411E182F8C859D850E941F1EE6
:103E600008C0C3010E94411E182FC3010E941F1EDB
:103E700000E04DE557E2612F110F770B6E0D711DBC
:103E800064197509002E000C110B282FC8018F0D25
:103E9000911DF7FC9A950E94B71A8DCFC4010E941C
:103EA000631E082FC4010E94411E182FC401D6CFE3
:103EB000EA85FB85838110E000E04CE057E2DBCF30
:103EC000A885B98511968C91883060F409E010E0DE
:103ED00046EA55E2833078F2835010E000E047E094
:103EE0005FE1C9CF883049F0893009F064CF10E133
:103EF00009E080E04EE552E2BECF10E100E080E054
:103F00004DEE51E2B8CFEE81FF81808110E000E0FC
:103F100040EF54E2B0CFAC81BD818C9110E000E065
:103F200046EA54E2A8CFF5018281882309F443CF01
:103F30009181892F880F890F20E0923008F4208129
:103F4000820F10E000E048EA53E295CF00E02AEA51
:103F50003EE144E953E26E2D70E064197509E12CED
:103F60008F2DFF0C990B0E94D71A25CF27E93EE130
:103F70004CE653E2F0CF00E010E04EE359E27BCF95
:103F800000E022ED3EE146EF56E2E5CF10E000E032
:103F900080E041E259E26FCF10E000E080E040E3D2
:103FA00059E269CF10E000E080E04CEE52E263CFCE
:103FB00000E026EE3EE14AE357E2CDCF00E02CEBF5
:103FC0003EE140EE56E2C7CFFC0184818F3060F4C1
:103FD0008D3070F48B3008F59381963279F050F47F
:103FE0009D3061F0A8F408958F30B1F789E008950D
:103FF00088E008959F3360F09F33A9F7818188237B
:1040000071F06AE00E94C53496E0981B892F0895EC
:104010008581883031F482E0089587E0089580E05A
:10402000089581E008952F923F924F925F926F9290
:104030007F928F929F92AF92BF92CF92DF92EF9238
:10404000FF920F931F93CF93DF9300D000D01F9266
:10405000CDB7DEB74C013B015C0129E7A20EB11CD4
:10406000D5011E96FC901C01B3EA2B0E311CF10108
:10407000808181110FC03896108111110CC0DB01B5
:1040800015968D919C9168E270E00E94D13411E008
:10409000853108F410E040E0B301C4010E94851EA0
:1040A0002401BDE64B0E511C6401ECE1CE0ED11C87
:1040B000C414D50401F1D60113968C91139788236B
:1040C000B1F016966C9116976F19062E000C770BAF
:1040D00015968C911597E12C12960C9129E53AE1F1
:1040E0004BE65AE1082E000C990B0E94D71AB9E052
:1040F000CB0ED11CDDCFCD82C40141960E94E41FBE
:10410000282FD4015596EC91559754968C9195EFA4
:104110009E0F953008F48150D4015B969C919923B1
:1041200009F440C0F0E0ED5DFF4EE491EF1963E06B
:104130006E0F062E000C770B90E02830A9F1293085
:10414000D1F1273009F03EC0E12C00E023ED39E148
:1041500045E15AE10E94D71AF1018081811107C01F
:10416000F401EC55FF4F8081882309F4F9C0D50193
:1041700012969C9112971C968C911C97911193C04A
:104180001F963C901F97311036C014969C9114973F
:1041900089131DC03324339416969C91943059F59D
:1041A000312C29C0E0E0C2CFE12C00E023E539E169
:1041B00042E959E1CFCFE12C00E02DEC38E14FE0AE
:1041C00059E1C8CF4FEA56E10E94B71AC5CF9817F8
:1041D0000CF055C0F50195819F5F958328E02683FB
:1041E000903109F41582D50115963C903694369499
:1041F000330CB3E03B0ED50114968C9314976D915C
:104200007C91C5010C960E94E11DF5018485E28137
:10421000F0E0E35AF44EE491D5011D966C911D97A0
:104220001E969C91691B6E1BB2E1B31508F448C041
:10423000E0E13E1608F44DC0F0EF3F0E30E020E024
:1042400047E755E1F401EC55FF4F90819A509B35BB
:1042500030F4D30153969C91992309F4A8C011110D
:104260007FC0062E000C770B082E000C990B211531
:10427000310509F071C0232D0E94B71A71C089174A
:104280000CF0B9CFF50195819F5F958324E02683DB
:10429000903109F41582D50115963C9036943694E8
:1042A0003394330CA8CFF5019481891379CF96818B
:1042B0002AE0322E943009F49ECF9BE0392E9BCF1A
:1042C000F4E1F31508F041C030E020E050E040E0B8
:1042D000B9CF643209F05BC193EF980F9F3308F0B8
:1042E00056C124E0321639F0231510F1332019F0AD
:1042F00092E0391226C090E049E454E1482E880F3C
:1043000055088BEFC82EE12C10E000E020E063E2BE
:1043100070E0F201E90FF11D97FDFA95CF010E94BF
:104320009818232D4DEC55E164E270E0C201A4CF52
:10433000A8E03A1601F3BAE03B16E9F2E6E03E16D1
:10434000D1F29FEF4BE554E1D9CF2DEE320E30E0A4
:1043500020E04DE455E176CFE32C032D0E94D71ADF
:10436000F3018289813099F54D805D2C4A145B04FC
:1043700071F1D2018C918823B1F015960C911597AB
:1043800014966C9114976F19062E000C770B1396E8
:104390008C91E02E29EE32E14DE653E1082E000C1F
:1043A000990B0E94D71AB6E04B0E511CDFCFF401D7
:1043B000EB55FF4F20812F3F99F22150062E000C24
:1043C000770B43EF53E1082E000C990B55CF40E4D7
:1043D000B301C4010E94851EF30183898111B9C014
:1043E000F401E655FF4F8081882309F4BEC0E12C1B
:1043F00000E02BE832E149EB52E16EE170E082E04F
:1044000090E00E94D71AD30151961C91812F64E647
:104410000E94C534282F41E652E167E270E086E051
:1044200090E00E94B71A2AE0812F622F0E94C534C3
:10443000192F0E94C534292F41E652E167E270E04E
:104440008BE090E00E94B71A212F41E652E167E22B
:1044500070E080E190E00E94B71AE12C00E02BEFC1
:1044600031E14DE252E170E060E086E690E00E94CA
:10447000D71AD30150968C91833050F029EE31E158
:1044800041EF51E16AE070E086E690E00E94D71AC1
:10449000F3018089823060F0E12C00E029EE31E107
:1044A00041EF51E16AE070E08EE690E00E94D71A99
:1044B000D30150968C91882361F0E12C00E029EE25
:1044C00031E141EF51E16AE070E086E790E00E945F
:1044D000D71A19821A821B821C82F301868597855E
:1044E000FE0131966E0125E0C20ED11C2AE030E0BB
:1044F000B9010E94D1348193CB01CE16DF06C1F7FA
:1045000009E610E0D6012E916D014FEB51E163E019
:1045100070E0C8010E94B71A0B5F1F4F0D371105DD
:1045200089F70F900F900F900F900F90DF91CF9120
:104530001F910F91FF90EF90DF90CF90BF90AF90C1
:104540009F908F907F906F905F904F903F902F90B3
:104550000895E12C00E025ED30E149E451E168E106
:1045600070E083E290E00E94D71AF40182818823F0
:1045700009F473CFE12C00E023E330E143E850E19C
:1045800068E170E08CE290E00E94D71A66CF2DE6D9
:1045900034E14DEC55E156CEFC018381843051F07D
:1045A0008830A9F081818350853018F484818D5F33
:1045B000818308958481882329F0853098F781507C
:1045C0008483F0CF81E0848388E08383EBCF848190
:1045D000843028F0843031F793E09483F6CF8F5FF6
:1045E000EFCFDC0183E0689FB0011124FB01E754A9
:1045F000FF4F9491FB01E654FF4F849165547F4F28
:10460000FB0164919C9311968C931197862F877070
:1046100013968C93139770E083E0759567958A9550
:10462000E1F712966C9308950F931F93CF93DF9346
:10463000EC016C968C0103591F4F0C171D0769F094
:1046400088818C3940F0188260E0CE0105960E9486
:10465000F1221B821C822996F0CFDF91CF911F910E
:104660000F9108952091AD02E091AB02F091AC0260
:10467000CF0102969093AC028093AB02222319F0F3
:10468000859194910895808191810895E1E7F0E00A
:1046900080818D7F80831092910046984798109278
:1046A0008B0208951F93CF93DF93EC01162F83E8BD
:1046B00084BD8FEF87BD81EF8093800010928800CA
:1046C00010928A000E9446231883DF91CF911F9198
:1046D0000895EF92FF920F931F93CF938C017B016C
:1046E000FB01C085C0958781C823F80181898F317E
:1046F000D8F0FB018581968180FD16C0F8012289E2
:10470000263290F42F5F228B83709927892B61F4D6
:104710008489823018F58F5FF801848B8389882320
:10472000F9F08150F801838BC3FD1CC081E0C2FD0C
:104730001AC0C7FD02C0C07629F065E0C7014596E2
:104740000E945223F8018189823810F48F5F818B97
:10475000CF911F910F91FF90EF90089580E0DCCFF3
:1047600082E0E0CF80E0F701828B64E0C7014596EC
:104770000E945223DECFCF92DF92EF92FF92CF932F
:10478000DF930E943223811520E8920741F4DF91E4
:10479000CF91FF90EF90DF90CF900C94462321E0D3
:1047A00020938B02813020E8920751F480919B0284
:1047B00090919C029093AC028093AB020E943223B2
:1047C00097FD05C020918E02222309F45BC0209141
:1047D0008F02211157C021E020938402EC01DF7782
:1047E000209709F052C081E08093860246984FE9F5
:1047F000C42E4FE0D42EE12CF12CCAEFD0E0E09192
:104800008C02F0918D020995811103C081E08093A3
:10481000860280918402882329F080918602882371
:1048200009F456C047980E943223009709F454C0F7
:104830009C01DE010E94B634DC01CB0129E0B59574
:10484000A795979587952A95D1F7109290002AE021
:1048500020939100D0929900C09298008093870293
:1048600090938802A0938902B0938A02809171008C
:10487000826080937100DF91CF91FF90EF90DF9085
:10488000CF90089510928402A9CFCF3F8FE7D80729
:1048900061F41092860281E08093850230ECC32E91
:1048A00031E1D32EE12CF12CAACF9E0150E040E063
:1048B00060E472E48FE090E00E94623469017A0162
:1048C00081E0C81AD108E108F1081092860297CF5A
:1048D0004699A8CF479AA7CF8FEF9FEFDC01B5CFBE
:1048E0009C01E1E7F0E090819D7F90831092AD0202
:1048F000EDE9F2E0F093AC02E093AB02F0939C029E
:10490000E0939B02318320838EE190E09383828346
:1049100080E090E8958384830C94BB230F931F93CE
:10492000CF93DF93EC018B01FB018085809597810C
:10493000892391F08989882311F084E1898B898901
:1049400081110DC08EE690E00E9470248CE290E010
:104950000E94702481E0898B8989882369F08F5FA8
:10496000898B853149F462E0C8014596DF91CF918A
:104970001F910F910C945223DF91CF911F910F91B2
:1049800008959C01E1E7F0E090819D7F908381E0B4
:104990008093AD023093AC022093AB0230939C0223
:1049A00020939B020C94BB23FC01DB0183E0509617
:1049B0008C9350971F961C921E921E9781E05196E1
:1049C0008C93519753961C9223E53BE130938D02D3
:1049D00020938C0210928F0210928E0280938F028D
:1049E00084E0828B138A148A118A8CE59AE20C94F3
:1049F000C1240895EF92FF921F93CF93DF9300D0CD
:104A000000D000D0CDB7DEB764E485EC91E00E9421
:104A100042346BE486EC91E00E94423487ECE82E4D
:104A2000FF24F39411E41A8219821E821D821B83D3
:104A30001C831D8346E050E0B701CE0101960E9421
:104A400032341F5F86E0E80EF11C8BEEE81681E041
:104A5000F80649F726960FB6F894DEBF0FBECDBF15
:104A6000DF91CF911F91FF90EF9008953F924F9269
:104A70005F926F927F928F929F92AF92BF92CF92EE
:104A8000DF92EF92FF920F931F93CF93DF93EC018E
:104A9000635F7F4F8C0100571F4FD80112967C93A4
:104AA0006E93119787589F4FFC0173876287B19669
:104AB000728361837A8F698F9E0126573F4F1596C7
:104AC0003C932E9314970E94091EFE01E956FF4F56
:104AD00081E0828374968083329783E480837E01B1
:104AE000F8EAEF0EF11C84E0D7018C93FE01EC553F
:104AF000FF4F89EC8083F801138210820480F581D6
:104B0000E02D82E0828384E18083FE01E655FF4F41
:104B100010826E01F3EACF0ED11CD6011C92CE0199
:104B20000E94F01B045711095E01BDE6AB0EB11CDB
:104B3000A016B10681F0F801108260E0C801059668
:104B40000E94F122D80113961C92139714961C927E
:104B5000075F1F4FEDCF912C8BE4482E512C612C19
:104B6000712C99E0892E33243394F70180819816B3
:104B7000F0F4A92CB12C0E94BC33A30192010E9435
:104B80006234645CD7012C91FE0190E0291739F161
:104B9000991631F0848D681730F4861B8E3058F3E7
:104BA0009F5F3996F3CFB62FB81B8B2FF7CFF60147
:104BB000108285E0D7018C931A82DF91CF911F91EB
:104BC0000F91FF90EF90DF90CF90BF90AF909F90AC
:104BD0008F907F906F905F904F903F9008958A9C48
:104BE00080018B9C100D11240C0F1D1FF801648F88
:104BF000CE01989C800D911D112481960E94F12276
:104C0000D8015F963C929394B0CF2F923F924F92EF
:104C10005F926F927F928F929F92AF92BF92CF924C
:104C2000DF92EF92FF920F931F93CF93DF93CDB755
:104C3000DEB766970FB6F894DEBF0FBECDBF8C010E
:104C40001B01DB0117965C9017971896BC91BA8BE5
:104C5000FC01828198012D553F4F398728878111AA
:104C60000AC6780139E7E30EF11CD70117968C913B
:104C7000811101C6E885F9858081882309F49CC0EB
:104C8000DB0115968D919C9180FD5EC7F701228115
:104C90002111D2C03085218531115DC721115DC739
:104CA0008089F52DF074CF2E282F2074D22E86FF08
:104CB0001CC055FE05C082FF03C0C7010E948030A2
:104CC000CC2089F0D70150968C91509783FF0BC070
:104CD0006D917C911197615071096D937C93C7011F
:104CE0000C960E94E11DD52C37C0FF2331F053FEF6
:104CF00002C087FD04C083FD7EC0D52C06C081E0C4
:104D0000F7018087C7010E948030D5FE25C0F701DA
:104D1000808982FF0AC0608171816150710971834D
:104D20006083C7010C960E94E11DF701808985FF11
:104D300013C0F801E057FF4F838181110DC081E05E
:104D400083839CE8908336971582828384E18083F5
:104D500088E59DE10E94C124D4FE11C0D701509680
:104D60008C91509781FF0BC06D917C911197615090
:104D700071096D937C93C7010C960E94E11DD7FECB
:104D800007C0F701808980FF03C0C7010E948030FF
:104D9000F801EA55FF4F808181110EC0D3FE0CC08F
:104DA000D70150968C9184FF07C083EA9AE10E9454
:104DB000C12481E0F7018283F701A684D101159611
:104DC0008C9180FD50C16801BAE8CB0ED11CF60170
:104DD0008581811148C19281923009F474C1933068
:104DE00009F491C1913009F03EC18081882309F412
:104DF00033C181505AC1D7018D919C91119784394B
:104E00009105B1F481E019968C9319978AED90E0A1
:104E100011969C938E9312961C926AED70E0C701D6
:104E20000C960E94E11D82E69DE10E94C12465CF9F
:104E3000C7010E94803061CF243218F42F5F228393
:104E4000BBCF1282B9CFD7018D919C918E3E910537
:104E500031F5B101C8010E940D1CAECFE59FF001F4
:104E60001124E85EF44EE491E93009F0AEC63C93BB
:104E7000ACC6E59FF0011124EC50F54EF4CFE59F50
:104E8000F0011124E155F54EEECF853A910509F474
:104E900097C008F4BEC0883A910509F499C0C701CB
:104EA0000E94803089CF893D910599F280F4873B3B
:104EB000910509F499C0873C910509F4B1C08E3A77
:104EC000910569F7C7010E94803089E07DC0833376
:104ED000B1E09B0709F4BBC08A33E1E09E0709F407
:104EE0009FC087329140D9F6F10186859785C29699
:104EF0009787868781898F5F818BC7010E94803069
:104F0000F801E855FF4F8081893010F48F5F80836E
:104F1000F801E755FF4F6081693508F04DCF6E5FAE
:104F2000608370E088EE93E00E94E534D101199629
:104F30006C9342CF233010F0421788F488EC90E055
:104F4000F70191838083128268EC70E0C7010C96B0
:104F50000E94E11D82E69DE10E94C1242DCFC70180
:104F60000E94803084E0D60111968C93119781E0E5
:104F700015968C9321CFC7010E948030F6011182D3
:104F800081E0D8015B968C935B9784E651968C9375
:104F9000519752961C92529753961C920DCFC7016F
:104FA0000E94803081E0F6018183F801E656FF4FD0
:104FB0008081882311F08150808387E39BE1CCCFEF
:104FC000C7010E94803082E0D60111968C93F4CE06
:104FD000C7010E94803085E0F6018183EDCEC701D4
:104FE0000E94803088E0F0CFF801E656FF4F8081C4
:104FF000811155CF80EF90E0F70191838083128279
:1050000060EF70E0C7010C960E94E11D82EB9CE10D
:10501000A3CFF101868597854496978786873FCFF2
:1050200088ECF801EC55FF4F80837497138210824F
:105030000480F581E02D82E0828384E18083F801A1
:10504000E655FF4F1082A885B9851C92B5CEF801B0
:10505000E956FF4F128223CFD6018181883039F182
:10506000F0F4833048F5F8017196FD87EC87D8019C
:1050700054968C91863209F464C58F3309F44CC080
:10508000D12C8D3009F44AC0863231F0C12CDD2498
:10509000DA948F3309F04BC0DD24DA943FC08930B5
:1050A00011F788E0F601818384E18083DCCF85E01D
:1050B000818384E18C93D7CF82E084838AE08083EC
:1050C00083E08283D0CF20818181222361F021502F
:1050D00020838350853038F68481823021F2C601E6
:1050E0000E94CC22C0CF883061F018F48330C8F61B
:1050F000BACF893009F0B7CF94838AE080831282D7
:10510000B2CF89E0CFCF8081811173CEC6010E94DA
:10511000CC228AE0D601CECF42E0D42EF80183899A
:10512000811104C0CC24C39482898111C12C0E94B6
:10513000BC339801245E3F4F3D832C8338013DE60C
:10514000630E711C23E030E040E050E00E946234C6
:10515000623071058105910589F5CC2081F1EC81E2
:10516000FD8190E0E615F70559F18381882321F14F
:105170009F5F80818E3400F52181D212C12C8B3348
:1051800048F08334C8F4D21217C0DD2061F08632B3
:1051900098F406C08E3148F0863270F4D2120CC0FA
:1051A00041E0D41209C0C12C07C0883028F4D212C3
:1051B00003C052E0D516B9F33996D4CFC12C90E094
:1051C000F801E855FF4F8081981768F5CC2059F118
:1051D000CC80DD806C147D0431F1D60113968C9166
:1051E000139781110FC114968C9181110BC10E94EC
:1051F000BC3323E230E040E050E00E9462346B5F59
:105200007F4F8F4F9F4FF6016483D8015896DC92F1
:10521000CE92579752961C92529753966C935397EF
:10522000645C51966C93F1018581968166E070E033
:105230000E94D134892B09F02EC1CC80DD809801E9
:105240002D553F4F3F872E87480139E7830E911C2C
:105250004A2D50E0598B488BB401645F7F4F7E8BA1
:105260006D8B6C147D0409F416C1D60113968C91D4
:10527000882309F4C3C0EE85FF858081882309F463
:105280004CC0D40112968C91882309F446C0F601D3
:10529000F581FC8BD6011696BC91BB8BF401608125
:1052A00071818D899E890E94E11DD4011296EC9135
:1052B000F0E0E35AF44EE491BC898B2FBB0F990BBD
:1052C000D4011C962C911C972817190631F51D96B0
:1052D0008C911D971E969C91891B8E1B082E000C8D
:1052E000990B2B892A19821B910927FD9395099700
:1052F000A4F4F6018181833080F42FEF2183D10162
:105300001E968D919C911F9701961F969C938E934C
:105310001E978CE99CE10E94C124D4011296EC9165
:10532000F0E0E35AF44E8491D10152968C91882397
:1053300009F46CC0813009F487C0AE85BF858C91BB
:105340008823B1F1E491D4011C968C911C97082E0E
:10535000000C990B9C01295F3F4F4A855B854217E2
:10536000530734F59A012B0D311D8217930704F56D
:105370001D968C911D971E969C91891B8E1B082E45
:10538000000C990B9C01255F3F4F6E817F81621756
:10539000730774F49B01240D311D8217930744F4A5
:1053A000B101C8010E940D1C8EE79CE10E94C1243E
:1053B000D6016C9117968C911797680F6F5F6C935D
:1053C000C60105960E94F122F6018581811105C072
:1053D0008681811102C010821382D60118968C91A9
:1053E0001897813009F44FC0823041F412968C91A5
:1053F000823008F046C08F5FF6018283F9E0CF0E5D
:10540000D11C2FCFB9E0CB0ED11CE4CED60115961E
:105410008C911597082E000C990B9C012E5F3F4F25
:105420003B872A8716968C91082E000C990B488989
:105430005989841B950BBC016E5F7F4F7F836E8300
:1054400035E0B32E4B2C79CFD60115968C9115975C
:10545000082E000C990B9C012F5F3F4F3B872A873A
:1054600016968C91082E000C990B48895989841B3B
:10547000950BBC016F5F7F4F7F836E8327E0B22E59
:10548000E1CF80E0B9CF12968C91882311F0815042
:10549000B3CF82E0B1CFD10152968C915297813037
:1054A00009F082C015968D919C916AE070E00E948F
:1054B000D134892B09F078C0630193E0492EF801BB
:1054C000ED55FF4FFF83EE834801F9E78F0E911CE6
:1054D000B12CEC14FD0409F467C0D6018C9188232B
:1054E00009F45EC011962C9111972F5F11962C93A1
:1054F000249D90011124F901EE57F44E8491F90195
:10550000ED57F44EA4912C57344EF9012491F60135
:105510008383A4832F712583811104C0A11102C04C
:1055200010821182EE81FF8190819923C9F1082EAA
:10553000000C990BF4012281E22FF0E0E35AF44EC3
:1055400024912A87F4012485022E000C330BB90123
:10555000695F7F4FAC014F5F5F4F4617570704F5F8
:10556000459628173907E4F4B0E0AA19BB098585E8
:105570009685891BFA858F1B082E000C990BAC01B0
:10558000455F5F4F9D012C5F3F4F2417350744F463
:1055900018968A179B0724F4B101C8010E940D1CBC
:1055A00026E0C20ED11C95CFD10152968C9181304C
:1055B00009F05CC05801BDE6AB0EB11C6801E3E721
:1055C000CE0ED11CD5018C91F6019081890FF3018B
:1055D00090E0EE16FF0649F02081222321F0218180
:1055E000921708F4922F3696F4CF882331F0813049
:1055F00009F03CC0933308F439C00E94BC3322E365
:1056000030E040E050E00E946234672B682B692B49
:1056100069F5D5018C91882309F461C0F601808178
:10562000882309F45EC08FEF980146E0849F200D27
:10563000311D1124C901F901E259FF4F1082E2E83E
:10564000FBE13491E3E8FBE12491E4E8FBE1E49140
:10565000DC01A059BF4F3C9311962C931196EF712A
:10566000EC93FC01E359FF4F81E08083D101159653
:105670008D919C9183709927892BC9F4F801E0578B
:10568000FF4F8081882399F0813069F51082138261
:105690000480F581E02D82E0828384E18083809123
:1056A0008B02811104C086E69CE10E94C124F801AE
:1056B000838D882381F184898632C0F48E3030F561
:1056C0008D30F9F0EC81FD816E167F0609F4AFC0D4
:1056D0008481882311F0815084833996F5CF80E04E
:1056E000A3CF81E0A1CF81508083E1CF873250F3F7
:1056F0008F3360F08F3331F784E0868B8EE3848BB9
:10570000E1CF88E0868B8EE0848BDCCF8C859D8515
:105710000E94281CD7CF8389882369F08150838B0E
:10572000811102C088E2828BF80181898823E1F12E
:105730008150818BC7CFD288DD20B1F3DA94D28A31
:10574000D110F2CF8489863249F18F3351F1D801DB
:105750005796ED90FC908091040190910501A091E5
:10576000060189839A83AB83FE01ED0DF11D6181F2
:10577000F7016083C70105960E94F122D7011196B7
:10578000DC92119781E013968C9380918B028111AA
:10579000CBCF80E79CE10E94C124C6CFDD24D39407
:1057A000D6CF82E0D82ED3CF8489863269F108F52E
:1057B0008D3031F108F486CF8C859D850E94281CA0
:1057C000D80154968C91863229F08F3319F08D30A0
:1057D00009F078CF0E94BC3322E830E040E050E08E
:1057E0000E9462346A5B7F4F8F4F9F4FF801618B3D
:1057F00069CF8F3308F38F3309F064CF84E001C0A1
:1058000088E0F801868BD8CF0E94BC3322E030E0DC
:1058100040E050E00E946234672B682B692B29F42A
:1058200084E0D80156968C93C7CF88E0FACFD10197
:1058300015962D913C91C90166E070E00E94D1342B
:10584000892B49F4F801EA56FF4F8081833008F034
:10585000A8C08F5F8083C9016CE070E00E94D134E2
:10586000892B49F4F801E956FF4F8081823008F016
:105870009AC08F5F8083F101808998012D553F4F39
:105880005901811104C091E0938BD9011C927801D8
:10589000B4EAEB0EF11CF701D080F8E2DF1609F450
:1058A000ECC0FD1508F48EC029E02D1508F47DC06C
:1058B00032E0D31608F0E7C041E0D41609F4E8C09E
:1058C000D7018C91882311F081508C936801B6EA3E
:1058D000CB0ED11CF6018081882311F0815080838A
:1058E000D10153969C91F50180818111F9C09111EC
:1058F000F7C08A8980958521F82FF870AF2E8C70BB
:10590000B9F1D7018C91853618F0C8010E94142393
:10591000BB24B394E885F985B082F801E655FF4FC2
:1059200010823597108236961082D7011C92C801DA
:1059300087589F4F0E94091EF801E057FF4F1382BE
:1059400010820480F581E02D82E0828384E18083EF
:10595000F801E956FF4FB282339680818111B7C0BA
:10596000C8010E94F01BAA2019F084E1D6018C9393
:1059700066960FB6F894DEBF0FBECDBFDF91CF9114
:105980001F910F91FF90EF90DF90CF90BF90AF905D
:105990009F908F907F906F905F904F903F902F904F
:1059A000089580E057CF80E065CF54E1D51609F423
:1059B00068C06EE1D61609F462C07AE0D71280CFD3
:1059C00081E00EC094E69D1578F0ADE3DA16E8F4B8
:1059D000B2E3DB1609F44FC0ECE386E0DE1270CFD1
:1059E000F801EB55FF4F0DC0F8ECFD1560F429EC04
:1059F000D21266CF8FEFF801EB55FF4F808381E025
:105A0000359680835DCF8FEFEBCF9FEFF801EB559D
:105A1000FF4F908391E035969083882309F450CF0F
:105A2000F19711821082128270E060E0CF010C9633
:105A30000E94E11DC8010E941423F801E656FF4FA1
:105A40008081811104C0C8010E94F01B39CFD801A8
:105A500051961C92519752961C92529753961C92B3
:105A600053978DE054968C9354975B961C925B975A
:105A700055961C9225CF85E0B3CF84E0B1CF83E06B
:105A8000AFCF82E0ADCFF801EB55FF4F108218CFBA
:105A9000882339F0C80187589F4F0E94091EF501DD
:105AA000D082F801EB55FF4F108236961082319765
:105AB0001082739781E08283D801A856BF4F8C91E2
:105AC000823018F48F5F8183FBCE80E0FCCFF80139
:105AD000118A128A138A8DE0848B138E158A43CF24
:105AE000F10180858095278182239923F9F083FF36
:105AF0003FCF65E0C101459666960FB6F894DEBFCC
:105B00000FBECDBFDF91CF911F910F91FF90EF900E
:105B1000DF90CF90BF90AF909F908F907F906F90CD
:105B20005F904F903F902F900C94522382FF20CF94
:105B3000D80112968C91129791E0892712968C9336
:105B400017CFDD24D394EACAD7011E96AC908BCA36
:105B5000F701A68438C9222341F0AC0143705527D0
:105B6000452B09F470C9332399F383709927892B46
:105B700079F7F101828943E0813009F044E0D701EF
:105B80008D919C916801BAE8CB0ED11CF601218160
:105B9000BC01605A71096732710530F57096308129
:105BA000311122C0D801A356BF4F53E03C91E1E030
:105BB000E30FEC9311966C911197613009F459C978
:105BC00008F44CC9623009F45AC91296688579857F
:105BD0006A177B0759F7D80155963C9155973F3086
:105BE00018F43F5F55963C938B3A910509F4F7C939
:105BF00008F059C9833A910509F4D1C908F045C99B
:105C00008839910509F496C98F39910509F4B3C90A
:105C10008739910509F043C9243008F440C9421777
:105C200008F43DC981E0D60115968C93C7010E9406
:105C3000803035C9CF92DF92EF92FF920F931F937E
:105C4000CF93DF93EC01DB0117961C9117978B8D97
:105C5000FE01811198C07C962F892F3F09F498C0CE
:105C600015968D919C916CE070E00E94D134892B47
:105C700009F06EC046E0249FE00DF11D112432961C
:105C800017FF19C0A88DAE0FBF2FB11D8C918F5F6C
:105C90008C93A88DAE0FBF2FB11D8C918B3514F056
:105CA00081E48C93A88DAE0FBF2FB11D8C918034F1
:105CB00011F481E48C9314FF10C0A88DAE0FBF2F98
:105CC000B11D8C9181508C93A88DAE0FBF2FB11D4B
:105CD0008C91813414F48AE58C9315FF05C0888D6E
:105CE000882311F08150888F16FF05C0888D82307F
:105CF00010F48F5F888F13FF2BC080818F3341F1A9
:105D000081818F3329F182818F3311F16F0182E01C
:105D1000E82EF12C06E0F60161916F012F898B8D41
:105D2000811133C087EC91E0A701209F400D511DE8
:105D30001124840F951F0E9442345FEFE51AF50A83
:105D400085E0E816F10439F78FEF8F8B84E68A8FB0
:105D5000898D1076103609F063C08F5F898F853189
:105D600020F08D3358F18D33E1F18A8D882311F0C5
:105D700081508A8FDF91CF911F910F91FF90EF900B
:105D8000DF90CF900895BE9667CF89ED91E0CCCF9C
:105D900018969C911897909591239C7041F08A8D4C
:105DA000811105C062E0CD0145960E94522315FD88
:105DB0001B8E16FFCDCF81E08B8FCACF20E430E061
:105DC000F901E81BF109CF01880F93E894BD9FEF1B
:105DD00097BD91EF909380001092880080938A0085
:105DE000C4CF198E83E884BD8FEF87BD81EF809388
:105DF00080001092880010928A000E94FA2442E1EA
:105E000050E067EC71E0CE014C960E94143442E100
:105E100050E069ED71E0CE018E960E941434A5CF5A
:105E2000882309F4A2CF83E884BD8FEF87BD81EF7B
:105E3000809380001092880010928A00198E95CF6E
:105E40003F924F925F926F927F928F929F92AF920A
:105E5000BF92CF92DF92EF92FF920F931F93CF9357
:105E6000DF9300D000D000D0CDB7DEB78C017B012E
:105E70008EE0FB018187F801108E118E84E6828FFF
:105E8000FB018289F801838FFB01668477846114AA
:105E90007104D1F139EDA32EBB24B394811104C058
:105EA00027ECA22EBB24B3946501512CC6010E949D
:105EB0002C346816790608F14501FCE08F0E911C20
:105EC00082E0482E96E0392E541408F54A94B50124
:105ED000439C600D711D112446E050E0CE010196F7
:105EE0000E94143446E050E0B401CE0101960E94B5
:105EF0003234F6E08F1A9108E7CF539486E0C80E4B
:105F0000D11CE3E05E12D2CF55245A940FC01E82FA
:105F10001D828FE38B838C838D837A82698246E036
:105F200050E0B601CE0101960E943234F801578A42
:105F3000F7011086178242E150E067EC71E0C8017A
:105F40004C960E94143442E150E069ED71E0C801C2
:105F50008E960E94143426960FB6F894DEBF0FBEBC
:105F6000CDBFDF91CF911F910F91FF90EF90DF9008
:105F7000CF90BF90AF909F908F907F906F905F90E9
:105F80004F903F9008950F920FB68F939F93EF938A
:105F9000FF93809192028D5F8D3708F08D5780932B
:105FA0009202E3E9F2E080818E4F808391819F4FDE
:105FB000918382818F4F828383818F4F8383E7E92F
:105FC000F2E080818F5F808381818F4F8183828126
:105FD0008F4F828383818F4F83838FB18F606699C8
:105FE0001C9B88278F3681F480919102981B9630F4
:105FF00068F0E0E0F8E087E78083818388E18093C0
:106000006000F0936000FFCF90939102FF91EF91B9
:106010009F918F910FBE0F9018951F920F920FB600
:106020000F9211242F933F934F935F936F937F931E
:106030008F939F93AF93BF93EF93FF9380918702CA
:1060400090918802A0918902B0918A02892B8A2BB3
:106050008B2B09F44DC080918602811118C080916C
:106060008502882349F080919800909199000F97BC
:10607000909399008093980088B190E4892788B91B
:1060800080918402882319F088B1805888B9809162
:10609000870290918802A0918902B0918A02181615
:1060A00019061A061B069CF48091870290918802BB
:1060B000A0918902B0918A020197A109B109809348
:1060C000870290938802A0938902B0938A02FF917D
:1060D000EF91BF91AF919F918F917F916F915F9160
:1060E0004F913F912F910F900FBE0F901F901895D9
:1060F000809185028111109285020E94BB23E7CF17
:10610000FC01608171816F5F7F4F718360830C96AA
:106110000C94E11DCF93DF93EBE5F1E0178210863D
:1061200080E181871682158213868BE391E0938349
:10613000828380E090E89093AA028093A902469817
:106140003E9A47983F9A17861686C1E0C08BC18B4E
:10615000128A138A108EC18F128E8FE291E0978B74
:10616000868B17A210A611A612A615A6C6A717A65B
:1061700083E291E094A783A714AE17AEC0939B016E
:1061800010929C0187E191E096AF85AF88E2809301
:10619000A9011092AA011092AB018DE08093AC018D
:1061A0001092AD011092B3011092050210920602F6
:1061B0001092070210920B0210920C0210920D0224
:1061C000D8E0D09317021092180210921902109280
:1061D0001A0210921202109211021092130270E031
:1061E00060E08DE192E00E94E11D1092220289E0C0
:1061F0008093230210922402D093250282E08093A0
:1062000026021092280210922B0210922E02109257
:106210002F0210923002C093310284E08093320248
:106220001092350210923602109237021092380204
:106230001092390210923A0210923B028BE0809346
:106240003F021092400283E480934102C0934202D5
:10625000C093430210924602C09347021092480234
:106260008BE091E090934502809344021092550296
:106270008FE2809356028EE5809357021092580267
:106280001092590210925A0210925B0210925C0214
:1062900010925D0284E680935E0210925F02DF91AD
:1062A000CF910895C1E0C093E0001092E2001092F7
:1062B000E10080E28093D8001092D70080916500C1
:1062C000806880936500789483E084BD83E085BD19
:1062D000C0936E00E1E8F0E083E08083E0E881E0D5
:1062E0008083E1E983E08083E0E981E08083E1EC81
:1062F00087E08083E3EC81E08083E0EC82E08083D0
:10630000E2EC81E08083EAE787E080838068808335
:10631000559A209A5D9A289A8C9A84988AE090E0FF
:106320000E94301B7C990EC0F89487E78093000888
:1063300080930108A89588E18093600088E08093AD
:106340006000FFCF81EC80937C0085B1806F85B9C0
:1063500084B1877E84B984B1876E84B95E9A5F9870
:106360008AB1806D8AB9769A6E9881B3806F81BB4D
:10637000899880B38D7080BB80E58CBDCDBD85E0F4
:1063800090E00E94301B5F9A85E090E00E94301BF5
:106390005E985C98ECEAF0E084918EBD00000DB44C
:1063A00007FEFDCF319600E0E93BF007A9F75C9AC4
:1063B00081E880936400809165008160809365002E
:1063C0000E944B1B87FF10C05C9885EA8EBD0000C1
:1063D0000DB407FEFDCF5C9A2E982F982D9881E082
:1063E00083BF889513BEFCCF0E944B1B82FF46C023
:1063F0002D980E944B1B84788438D9F42D9A88EC10
:1064000090E00E94301B2F9882E090E00E9424349C
:106410008F3F29F06FEF82E090E00E94543484EFC8
:1064200091E00E94301B2F9A0E944B1B8478843885
:10643000D9F30E944B1B84718431D9F42D9A88ECD6
:1064400090E00E94301B2E9882E090E00E9424345D
:10645000882329F060E082E090E00E94543484EFC9
:1064600091E00E94301B2E9A0E944B1B8471843154
:10647000D9F388EC90E00E94301BB6CF2D9A82E0D1
:1064800090E00E942434882309F474C03E9A3F9A15
:1064900081E080939002809164008E7F80936400FD
:1064A00080917A00806480937A0080917A0086FDE2
:1064B000FCCFC0917800D09179000E948018AB0188
:1064C000BC01CE01B0E0A0E0DC01992788278C0157
:1064D0009D01040F151F261F371FC901B801209108
:1064E00064002160209364006115710581059105A8
:1064F00011F00E940B348EE08093640185EC91E0F2
:106500000E942434C82F86EC91E00E942434C434C5
:1065100011F48B3411F00E94FA2481E08093700111
:1065200023E53BE130938D0220938C0210928F0281
:1065300010928E0280938F02C1E0D1E079010EEAC1
:1065400012E08FB7F89440919302509194026091B9
:106550009502709196028FBF80916501242F281BB0
:10656000822F90916601992351F020936701109238
:106570006601E7CF109290023E983F988CCF9091A1
:106580006401291738F48F5F8917D8F6C3BF88953F
:1065900013BED7CFD093660140936501809160010F
:1065A00090916101019690936101809360018091C7
:1065B0006201809363010E944B1B80936201809172
:1065C0007001823009F452C080F4813081F1F80109
:1065D00080E098E000800EBCC111012C019780FD85
:1065E000FDCF0192B9F70DB4ACCF843009F45BC094
:1065F000853069F790916F01953061F080935B0170
:106600006BE571E084E492E00E94202F809170019C
:1066100080936F016BE571E084E492E00E941A2E92
:106620006BE571E084E492E00E94361CD0CF90913B
:106630006F01913071F080935B01F0928D02E092D6
:106640008C0210928F0210928E0280938F028093A0
:106650006F016BE571E086E891E00E948E246BE5A6
:1066600071E086E891E00E94A61BB1CF90916F0186
:10667000923061F080935B016BE571E081E791E01E
:106680000E94D4248091700180936F016BE571E0CA
:1066900081E791E00E9469236BE571E081E791E079
:1066A0000E94571B94CF90916F01943061F08093BA
:1066B0005B016BE571E088E991E00E9436258091ED
:1066C000700180936F016BE571E088E991E00E94B1
:1066D00005266BE571E088E991E00E94132077CFF1
:1066E0008F929F92AF92BF92CF92DF92EF92FF92E2
:1066F000CF93DF93EC01688179818A819B81611559
:1067000071058105910521F464E279ED8BE597E04F
:106710002DE133EF41E050E00E94623449015A011B
:106720009B01AC01A7EAB1E40E9481346B017C01BA
:10673000ACEEB4EFA50194010E948F34C60ED71EB3
:10674000E81EF91EF7FE06C081E0C81AD108E1086C
:1067500080E8F80AC882D982EA82FB82C701B601C2
:106760009F77DF91CF91FF90EF90DF90CF90BF9018
:10677000AF909F908F9008958F929F92AF92BF920B
:10678000CF92DF92EF92FF92609100017091010130
:1067900080910201909103016115710581059105B8
:1067A00021F464E279ED8BE597E02DE133EF41E0F0
:1067B00050E00E94623449015A019B01AC01A7EAF2
:1067C000B1E40E9481346B017C01ACEEB4EFA50111
:1067D00094010E948F34C60ED71EE81EF91EF7FEE4
:1067E00006C081E0C81AD108E10880E8F80AC09222
:1067F0000001D0920101E0920201F0920301C70171
:10680000B6019F77FF90EF90DF90CF90BF90AF9051
:106810009F908F9008956093000170930101809381
:106820000201909303010895DC01CB01FC01F99969
:10683000FECF06C0F2BDE1BDF89A319600B40D92CC
:1068400041505040B8F70895F999FECF92BD81BDEF
:10685000F89A992780B50895A8E1B0E042E050E0A9
:106860000C941634DC01A40FB51F4150504048F081
:10687000CB01840F951F2E910E944334415050400C
:10688000D0F70895262FF999FECF92BD81BDF89AD1
:10689000019700B4021639F01FBA20BD0FB6F89464
:1068A000FA9AF99A0FBE0895262FF999FECF1FBACA
:1068B00092BD81BD20BD0FB6F894FA9AF99A0FBE29
:1068C00001960895052E97FB1EF400940E947934DA
:1068D00057FD07D00E94943407FC03D04EF40C946B
:1068E000793450954095309521953F4F4F4F5F4FEC
:1068F000089590958095709561957F4F8F4F9F4F2C
:1069000008950E94B634A59F900DB49F900DA49F4A
:10691000800D911D11240895B7FF0C9481340E94BD
:106920008134821B930B0895A1E21A2EAA1BBB1B74
:10693000FD010DC0AA1FBB1FEE1FFF1FA217B3074B
:10694000E407F50720F0A21BB30BE40BF50B661F61
:10695000771F881F991F1A9469F760957095809525
:1069600090959B01AC01BD01CF010895A29FB0019C
:10697000B39FC001A39F700D811D1124911DB29F73
:10698000700D811D1124911D0895991B79E004C09B
:10699000991F961708F0961B881F7A95C9F780955E
:1069A0000895AA1BBB1B51E107C0AA1FBB1FA61756
:1069B000B70710F0A61BB70B881F991F5A95A9F7A8
:1069C00080959095BC01CD01089597FB072E16F494
:1069D000009407D077FD09D00E94D13407FC05D080
:1069E0003EF4909581959F4F0895709561957F4FE6
:1069F0000895EE0FFF1F0590F491E02D0994F8948F
:026A0000FFCFC6
:106A0200010000003B1E0000000000202FF9241AA4
:106A12002E361C000000003625F92405261320001E
:106A2200000000E21BF9248E24A61B00000000D403
:0E6A320024F9246923571B00000000561B00A6
:00000001FF
